:046F1A00010001442D
:10698C00AF50055074D02FF582E4341DF583E59992
:10699C00F022D3E5309400E52F94002290000FE014
:0369AC006403225F
:0300030002569012
:0B569000C0E0C083C082C0D075D0080D
:10569B00852E82852D83E493FF201404C4540FFFC1
:1056AB00430FF08F80C284D28500C2870000D2875F
:1056BB00007580FF7580FEC284C28500C287000022
:1056CB00D287007580FF30140CC214052EE52E70A6
:0956DB0006052D8002D214D2A8AC
:0956E400D0D0D082D083D0E03296
:03000B0002195F78
:10195F00C0E0C0F0C083C082C0D075D008758CD8ED
:10196F00758A92D28C1242111262E0E531D3940043
:10197F0040171531E53164056009E531640F6003E7
:10198F00021B71126BD1021B71753114E54ED3948A
:10199F00004002154EE54FD394004002154FE53A33
:1019AF00D394004002153AE54BD394004002154BF7
:1019BF00154CE54C123A4A1B63001B38011B1002F1
:1019CF001AE8031A65041A4C051A33061A1A071A6D
:1019DF00010819E80900001B6ED3E52C9400E52BD4
:1019EF0094005003021B71E52C152C704D152B0222
:1019FF001B71D3E5379400E53694005003021B7139
:101A0F00E537153770021536021B71D3E548940080
:101A1F00E54794005003021B71E548154870021505
:101A2F0047021B71D3E54A9400E549940050030225
:101A3F001B71E54A154A70021549021B71D3E52A3D
:101A4F009400E52994005003021B71E52A152A70B2
:101A5F00021529021B717885E6FF7003021B71EFD7
:101A6F00B40105900524801BEFB4021012699E404B
:101A7F002FE53015307002152F021B71EFB4030CD8
:101A8F00900526E0F52FA3E0F5308028EFB404127F
:101A9F0012699E400BE53015307002152F021B7135
:101AAF008012EF64057003021B71EFB4060C752FE3
:101ABF0002753058788506021B71EF6407600302C8
:101ACF001B7112699E400BE53015307002152F0205
:101ADF001B7178857600021B71D3E5399400E538C8
:101AEF0094004008E539153970021538D3E53C9458
:101AFF0000E53B9400406BE53C153C7002153B80C4
:101B0F0061D3E5579400E55694004008E557155703
:101B1F0070021556D3E5559400E55494004043E503
:101B2F00551555700215548039D3E5359400E534B9
:101B3F0094004008E535153570021534301523D360
:101B4F00E5339400E53294004018E53315337012F5
:101B5F001532800EE551D394004004155180007565
:0D1B6F004C0AD0D0D082D083D0F0D0E0322C
:03001300023EDFCB
:0D3EDF00C0E0C0F0C083C082C0D075D0101C
:103EEC00E545C394504003023FA0202403023FA0A9
:103EFC00300C03023FA0E5A0540FF5587D077F015D
:103F0C00124ED25067202364E545700DE558B40C71
:103F1C0008201105D211023FA020034A201147129C
:103F2C003FAB50047F0180027F0F126E9D90000FFB
:103F3C00E0FF64016012EFB40302800C90000FE00C
:103F4C00B40209123FAB50047F80801290000FE046
:103F5C00B4020E7D037F07124ED240057FA01200E3
:103F6C0016754202D20390053CE0F53A90002BE026
:103F7C00B5580D7D087F05124ED25004D226801400
:103F8C00053EE53EAE3D7002053D14F5828E83E59F
:043F9C0058F005458F
:103FA000D0D0D082D083D0F0D0E0327D037F071212
:033FB0004ED222CC
:030023000263B9BC
:1063B900C0E0C083C082C0D075D018309819C29887
:1063C900E599B40A0812698C755000800AE550C332
:1063D9009490500312698C309902C299D0D0D0821E
:0563E900D083D0E0327A
:03003B0002491D5A
:0D491D00C0E0C0F0C083C082C0D075D018CB
:10492A00C2CEE546C39410507C302579200C76AF70
:10493A00A07804EF08800123D8FDF55953590F7D5B
:10494A00077F02124ED25035202332E546700CE51D
:10495A0059B40C07201304D213804A2004192013D7
:10496A001690000FE0B4020F7F0A126E9D7F80122C
:10497A000016754202D20490053CE0F53A90002BED
:10498A00E0B5590D7D087F05124ED25004D2288019
:10499A00140540E540AE3F7002053F14F5828E8350
:0549AA00E559F005468F
:0B49AF00D0D0D082D083D0F0D0E03216
:104B7C00E4F55AF55B755C1E755DFF855B82855AA5
:104B8C0083E0F55E635EFFE55EF0E0655E60031258
:104B9C006F1E635EFF855B82855A83E55EF0E06580
:104BAC005E6003126F1E055BE55B7002055AE55DE6
:104BBC00155D7002155CD3E55D9400E55C940050C6
:104BCC00BA75985A758921758845758DE7758780F2
:104BDC00758CD8758AEF75C90275C808753D1E7538
:104BEC003E60753F1E7540B075B701D2A9D2E8D2B0
:0F4BFC00AA75C64C75EEFF75FEFFD2AF12668923
:014C0B002286
:026F1E0080FEF3
:10696900202F0F90053AE0F54EE54ED394004012E2
:1069790080F7302F0D90053AE0F54FE54FD394009D
:0369890050F922A0
:1069210030310AD215900024E04420800DC2157F39
:1069310008126EDE900024E054DFF0FD7F247E001B
:046941001263832238
:102EB6008F70E570640170292030047F01805620F0
:102EC6003003022FB1122FC24003022FB1122FCAB4
:102ED600500C122FB2301503022FB1022FA7022F6A
:102EE60067E570640270202030047F02802720305E
:102EF60003022FB1122FD24003022FB11269A8701C
:102F060003022FB1022F81E57064036003022FB123
:102F16002030057F03026EDE303024122FC2501F90
:102F2600122FD2501A1269A86015122FCA500B7FA1
:102F36000B122FDA201574022FA77F03022FAE3053
:102F46003023122FE8501E7D017F02124ED240150B
:102F56007D017F07124ED25008122FB220154C80E9
:102F6600407F018043303017122FE840127D017FE9
:102F760002124ED250091269A860047F02802930DD
:102F860030297D017F01124ED250201269A8701B94
:102F96007D017F07124ED2500D7F09122FDA2015C0
:102FA6000AD2310269217F01126EF1227F09126E67
:102FB600F1900536E0F532A3E0F533227D017F017D
:102FC600124ED2227D017F07124ED2227D017F0250
:102FD600124ED222126EF1900536E0F532A3E0F5DC
:0A2FE60033227D017F01124ED2223A
:104C0C00C2957FFF126EDE124B7C7F07126317502A
:104C1C000512003E800312609ED28C7F081263172F
:104C2C0050051242D180FEC22B1268429000D1E096
:104C3C00FF7C117D00125BD8125D4B90000FE0B42D
:104C4C00010512281D801090000FE0FF6402600423
:104C5C00EFB40303123251123D1E301E11E54270A7
:104C6C000DE52754A060077FA0126E9DC21E7D0724
:104C7C007F05124ED24002C200E552C3940A50BBCB
:104C8C003015B8E533453270B2C23112692180ABB0
:104A5300EF253EFFEE353DCF2401FDE43FFC22AFC1
:104A63005A7E00EF2403FDEE33FC22E53E255AF582
:104A730082E4353DF58322E540255AF582E4353F4E
:104A8300F58322E56F256DF582E4356EF583E0FF4E
:104A9300E56F256DF582E4356EF58322E55A240230
:104AA300FFE433FE22E56C2401FFE433FEC3E56D2E
:104AB3009FEE6480F874809822EF2540FFEE353F27
:104AC30022C2017FF47E01126C27E56C25E0F56CB0
:104AD300756D0122E55C2EF582E4355BF583E0FD1F
:084AE30022753D1E753E6022A4
:106C2700EF1FAA0670011ED39400EA9400400BE4FC
:0A6C3700FDEDC394C850E90D80F78D
:016C41002230
:105169008F5BE55BB401197D017F06124ED2500CAD
:105179009000B1E0FF7C0D7D00125BD87885062296
:10518900E55BB402131251DB50439000B2E0FF7C9F
:105199000D7D20125BD88035E55BB404161251DB16
:1051A900500C9000B4E0FF7C0D7D60125BD87885CF
:1051B900760622E55BB403197D027F06124ED250B2
:1051C9000C9000B3E0FF7C0D7D40125BD8788576AA
:0A51D90001227D027F06124ED22251
:104ED200BF0107900020E0FE8048BF02079000213A
:104EE200E0FE803EBF0307900022E0FE8034BF0454
:104EF20007900023E0FE802ABF0507900024E0FE11
:104F02008020BF0607900025E0FE8016BF070790AD
:104F12000026E0FE800CBF0807900027E0FE80021A
:104F2200E4FEBD0103EE1322BD0204EEA2E122BDA6
:104F32000304EEA2E222BD0404EEA2E322BD0504B4
:104F4200EEA2E422BD0604EEA2E522BD0704EEA213
:074F5200E622BD0802EE3368
:014F59002235
:101D7D00124AE4900100E0F55A124A6EE0123A4A16
:101D8D001DAC011DE1021E16031E4B041E80051E17
:101D9D00B5061EEA071F1A081F460900001F70121C
:101DAD004A6EA3E0B40A15E55A124AA1E545B507F6
:101DBD000BE4B506077D017F01021F2E124A62E575
:101DCD00456D7001EC6003021F70124A53C2297FEA
:101DDD0001021F43124A6EA3E0B40A15E55A124AD6
:101DED00A1E545B5070BE4B506077D017F02021F8E
:101DFD002E124A62E5456D7001EC6003021F7012F0
:101E0D004A53C2297F02021F43124A6EA3E0B40A4D
:101E1D0015E55A124AA1E545B5070BE4B506077D50
:101E2D00017F03021F2E124A62E5456D7001EC60C1
:101E3D0003021F70124A53C2297F03021F43124A25
:101E4D006EA3E0B40A15E55A124AA1E545B5070B94
:101E5D00E4B506077D017F04021F2E124A62E54597
:101E6D006D7001EC6003021F70124A53C2297F048A
:101E7D00021F43124A6EA3E0B40A15E55A124AA195
:101E8D00E545B5070BE4B506077D017F05021F2E5D
:101E9D00124A62E5456D7001EC6003021F70124A33
:101EAD0053C2297F05021F43124A6EA3E0B40A15DF
:101EBD00E55A124AA1E545B5070BE4B506077D01C4
:101ECD007F06021F2E124A62E5456D7001EC60031C
:101EDD00021F70124A53C2297F06021F43124A6E17
:101EED00A3E0B40A14E55A124AA1E545B5070AE480
:101EFD00B506067D017F078028124A62E5456D70A3
:101F0D0001EC705F124A53C2297F078029124A6E75
:101F1D00A3E0B40A0F124A6EA3A3E070077D017F00
:101F2D0008024E47124A62E5456D7001EC7034129D
:101F3D004A53C2297F08020FF1124A6EA3A3E07023
:101F4D0022124A6EA3E024F96008147016E4FF0211
:101F5D005F287FF47E01126C277D5E7F0212665F23
:031F6D001242D14C
:011F7000224E
:101B7C00753F1E7540B0900108E0F55A124A7AE0A4
:101B8C00123A4A1BAE011BE6021C1E031C56041C17
:101B9C008E051CC6061CFE071D31081D66090000BB
:101BAC001D7C124A7AA3E0B40A13124A9FE546B58B
:101BBC00070BE4B506077D017F01021D49AF5A12E0
:101BCC004A64E5466D7001EC6003021D7C124ABC50
:101BDC00124A5AD2297F01021D63124A7AA3E0B439
:101BEC000A13124A9FE546B5070BE4B506077D01BB
:101BFC007F02021D49AF5A124A64E5466D7001EC32
:101C0C006003021D7C124ABC124A5AD2297F02027E
:101C1C001D63124A7AA3E0B40A13124A9FE546B533
:101C2C00070BE4B506077D017F03021D49AF5A126D
:101C3C004A64E5466D7001EC6003021D7C124ABCDF
:101C4C00124A5AD2297F03021D63124A7AA3E0B4C6
:101C5C000A13124A9FE546B5070BE4B506077D014A
:101C6C007F04021D49AF5A124A64E5466D7001ECBF
:101C7C006003021D7C124ABC124A5AD2297F04020C
:101C8C001D63124A7AA3E0B40A13124A9FE546B5C3
:101C9C00070BE4B506077D017F05021D49AF5A12FB
:101CAC004A64E5466D7001EC6003021D7C124ABC6F
:101CBC00124A5AD2297F05021D63124A7AA3E0B454
:101CCC000A13124A9FE546B5070BE4B506077D01DA
:101CDC007F06021D49AF5A124A64E5466D7001EC4D
:101CEC006003021D7C124ABC124A5AD2297F06029A
:101CFC001D63124A7AA3E0B40A12124A9FE546B554
:101D0C00070AE4B506067D017F078031AF5A124AF7
:101D1C0064E5466D7001EC7057124ABC124A5AD2F7
:101D2C00297F078032124A7AA3E0B40A13124A9F21
:101D3C00E546B5070BE4B506077D017F08024E4763
:101D4C00AF5A124A64E5466D7001EC7023124ABC1E
:101D5C00124A5AD2297F08020FF1124A7AA3A3E041
:101D6C00700E124A7AA3E024F870057F01125F28E6
:011D7C002244
:0447D0008C5B8D5C15
:1047D400055CE55C7002055B14F5828C83E0F9707E
:1047E40003024877EF7005124AE48009BF01067599
:1047F4003F1E7540B0302946EF7007E965456002F9
:10480400C322BF0107E965466002C322E4FEEEC38A
:10481400995029EF700F124AD7E53E2E124A72E0E2
:104824006D6002C322EF6401700F124AD7E5402E77
:10483400124A7EE06D6002C3220E80D2D322202968
:1048440033E4FEEEC3995029EF700F124AD7E53EC8
:104854002E124A72E06D6016C322EF6401700F12CB
:104864004AD7E5402E124A7EE06D6002C3220E80D4
:04487400D2D322C3B6
:01487800221D
:060FF1008F5BAB05AA04B2
:100FF7007D027F07124ED25011E55BB4050C8B8240
:101007008A83E06405700302125E7D017F07124E3A
:10101700D25011E55BB4050C8B828A83E0640670BD
:101027000302125EC22AEB24FFF582EA34FFF5833E
:10103700E0F55D8B828A83E0FFF55EA3E0F9F55F5B
:10104700EF123A4A106701106E02107503107C0404
:10105700108305108A061091071098080000109D4C
:10106700755C01D22A802F755C02D22A8028755CB4
:1010770004D22A8021755C08D22A801A755C10D2A6
:101087002A8013755C20D22A800C755C40D22A8096
:1010970005755C80D22AE924FE700302115F24F8EB
:1010A700605C24096003021171E55BB401059000DF
:1010B700208045E55BB40205900021803BE55BB4E9
:1010C70003059000228031E55BB40405900023807E
:1010D70027E55BB40505900024801DE55BB4060594
:1010E7009000258013E55BB407059000268009E58D
:1010F7005B64087077900027E0455CF0806EE55BE5
:10110700B401059000208045E55BB40205900021FD
:10111700803BE55BB403059000228031E55BB404B6
:10112700059000238027E55BB40505900024801D0A
:10113700E55BB406059000258013E55BB4070590D1
:1011470000268009E55B64087022900027E0FFE530
:101157005CF4FEEF5EF08014E55BB4050D8B828ACC
:1011670083E0FFD22F12297EC22AC22A202A030235
:10117700125EE55BB40109900020E0FD7F208060EE
:10118700E55BB40209900021E0FD7F218052E55B19
:10119700B40309900022E0FD7F228044E55BB4049C
:1011A70009900023E0FD7F238036E55BB4050990B5
:1011B7000024E0FD7F248028E55BB4060990002524
:1011C700E0FD7F25801AE55BB40709900026E0FD66
:1011D7007F26800CE55BB4080C900027E0FD7F2795
:1011E7007E00126383126D3CD2AF2029047F0180F9
:1011F700027F02126EF1A229922F126969AD5DE496
:10120700FF12665FAD5EE4FF12665FE55FB401043F
:101217007D388007E55FB40A077D367F0612665F73
:10122700E55BB405031264E77D077F05124ED250D4
:101237000A200007C2307F03122EB67D017F0112FC
:101247004ED24005C230122EB67D017F02124ED219
:071257004005C230122EB663
:01125E00226D
:024E47008F5B7F
:104E4900ED24FF922F126969E55B123A4A4E72010D
:104E59004E77024E7C034E81044E86054E8B064EDC
:104E690090074E950800004E9B90002080219000ED
:104E790021801C900022801790002380129000242A
:104E8900800D90002580089000268003900027E07F
:104E9900F55CE55C6024755E01E4F55DE55C30E098
:104EA90007AD5EE4FF12665FE55CC313F55C055E62
:104EB900055DE55DC3940840E3227D187F02126613
:084EC9005F7D537F0212665F5A
:014ED10022BE
:10631700C2AFD284C285BF070BC28600E580A2E266
:10632700922A8019BF080BC28600E580A2E3922A51
:10633700800BBF0508C28600E58013922AD286D259
:0563470085D2AFA22A7F
:01634C00222E
:1045BB00C229D22DE4FF1259B97D2E7F0312665FFB
:1045CB007D607F0212665F7F03126EDE3024FD205A
:1045DB0024FDE5456407703B7E017F50124AE48F52
:1045EB00828E837407F07D01E53E2D124A72E582BF
:1045FB0024FFF582E58334FFF583E0F9EF2DF58297
:10460B00E43EF583E9F00DBD08DED2297F647E0020
:10461B00126C277F081263175043302995D22DE473
:10462B00FF1259B97D607F0212665F7D327F0612E1
:10463B00665F7D1E7F0512665FC22DE4FF1259B9BE
:10464B007C017D507B087F507E011255057F08123F
:10465B00631750097F327E00126C2780F07F647ED7
:04466B0000126C27A6
:01466F002228
:02549C008F5A25
:10549E00900138E0F55BE55A7020E55B124AA1E514
:1054AE00456F7001EE704F7460255BF582E4341E1B
:1054BE00AF82F55D8F5E7F408024E55A64017036C1
:1054CE00E55B124AA1E5466F7001EE702974B025B6
:1054DE005BF582E4341EAF82F55D8F5E7F101200A5
:1054EE0016855E82855D83E0FFA3E0FD126D8A8FD7
:0654FE005CE4FD124F5AB0
:015504002284
:024F5A008D6B5D
:104F5C0075F020EF900280123A3EAF8285836E8FFF
:104F6C006FE0F56CD394004060E56C9410505AE5FA
:104F7C006B7014124AC6124AA8504E124A86124F2F
:104F8C00DB056D056D80EFE56B64017019124AC489
:104F9C00124AA85034124A86124FDB302402802960
:104FAC00056D056D80EAE56B6402701D124AC41232
:104FBC004AA85015124A86A3E0FD12651730240347
:0E4FCC00024D2B056D056D80E67F50126E9D27
:084FDA0022A3E0FD126517227D
:100D2400855C82855B83A3A3E0FF855C82855B830E
:100D3400A3222430F58274003EF583EDF0AF62EF18
:100D44003395E0FEE55F2FF582E55E3EF58322E50F
:100D5400822406F582E43583F583E0FF126D65ADE8
:100D640007AF63EF3395E0FEEF22A3A3E0FFE55C5A
:100D74002404F582E4355BF583E022E55F2405F580
:100D840082E4355EF583E022E55F2405F582E435EF
:100D94005EF583E0FFE55F2406F582E4355EF583C6
:100DA400E0228E69F56AAF68EF3395E0FEE5662FC1
:100DB400F582E5653EF583222455F582E4340AF58F
:100DC40083EFF0E56275F007A422AF60EF3395E09E
:100DD400FEE56175F008900158123A3EE5822FF560
:100DE40082E5833EF58322E5662405F582E43565D4
:100DF400F583E022E55E75F007A42454F582E4341B
:100E04000AF58322A3A3A3E0FF8D828C83E58224C9
:100E140004F582E43583F583E022E55E75F007A4EA
:100E24002451F582E4340AF5832224E0F582740A1D
:100E34003EF583E5822DF582E5833CF58322E55E6C
:100E440075F007A42453F582E4340AF58322E55FA0
:100E54002405F582E4355EF583E0FFE55F2406F5BD
:100E640082E4355EF583E022E55E75F007A4245242
:100E7400F582E4340AF58322749F2562F582E43412
:100E840000F58322746F2562F582E43400F5832231
:100E94002450F582E4340AF58322ECFF3395E0FE16
:100EA400EF25E0FFEE33FE75F02022E5602405F522
:100EB40082E4355FF58322D3EF6480948022AB070C
:100EC400AA068B828A83A3A3A3E0FFEB2404F58202
:100ED400E43AF583E0FD228F828E83A3A3A3E0226C
:100EE400855F82855E83A3A322AB5DAD5AAF5CAE02
:100EF4005B22FFE562FD3395E0FCE55F2DF582E5BD
:100F04005E3CF5832233CE33CE92E022A2E0CE13B0
:100F1400CE132275F00AA42DFDE5F03CFCE5662213
:100F2400E5602405F582E4355FF583E022E562752A
:100F3400F008900158023A3EE55E75F007A4245586
:100F4400F582E4340AF583E022AB5AAD5DAF5CAEC2
:100F54005B22EF7C002563FDEC35628D82F58322F4
:100F6400A3A3E0FFAD5A22540FF5657808AF03AE92
:100F740002EF08220564E564AE632275F020123A9C
:100F84003EE0FEA3E0FF22E0FAA3E0FB780CFFAE14
:100F9400020822E0FCA3E0FD7804FFAE040822E589
:100FA400632561F582E43562F58322E5662DF582D9
:100FB400E5653CF58322E5662FF582E5653EF5831C
:100FC400222431F5827400222480F58274023EAF1B
:100FD40082222560F560E4355FF55F2285608285B5
:0D0FE4005F83228F828E83A3A3E0640A2224
:02055B008F5AB5
:10055D00C22AE4F542D223D22D1259B97D4B7F0226
:10056D0012665F7D02E4FF12665F7D32E4FF126664
:10057D005F7D607F0212665F7D027F07124ED25053
:10058D00057F04126EDE900528E0F536A3E0F53701
:10059D007F03126EDEE55A7006A22492298009E5CA
:1005AD005AB40104A2259229E53745367005D22AA1
:1005BD00020A223029DFE55A7006A2249229800909
:1005CD00E55AB40104A22592292029EAE55A700BB7
:1005DD00755B1E755C6085455D800EE55AB401093D
:1005ED00755B1E755CB085465DE55DD3940050036B
:1005FD00020A1C855C82855B83E0640B6003020A42
:10060D0017A3E0FFB40A0AE55DB40205D22A020A77
:10061D001CEF6401701E120D2EA3E0640A7015E527
:10062D005D6405700F120D2E120D6E120A4D1231F2
:10063D0024020A1C120D2EE0B40111120D2EA3E09E
:10064D00B40109120EED12171B020A1C120D2EE039
:10065D006401701E120D2EA3E064027015E55D6439
:10066D0005700F120D2E120D6E120A4D12618C02B5
:10067D000A1C120D2EE06401701D120D2EA3E064F4
:10068D00037014E55DB4050F120D2E120D6EFDAB4A
:10069D005A123A70020A1C120D2EE0B4011D120DF1
:1006AD002EA3E0B40415E55DD39405400EAB5AAD11
:1006BD005CAC5BAF5D122FF0020A1C120D2EE064D4
:1006CD0001701D120D2EA3E064057014E55DB405D7
:1006DD000F120D2E120D6EFDAB5A125AF7020A1C97
:1006ED00120D2EE06401701D120D2EA3E064067034
:1006FD0014E55DB4050F120D2E120D6EFDAB5A12E1
:10070D004DBA020A1C120D2EE0B4011D120D2EA3BE
:10071D00E0B40715E55DD39405400EAB5AAD5CAC66
:10072D005BAF5D124670020A1C120D2EE064017063
:10073D001D120D2EA3E064087014E55DB4050F12B3
:10074D000D2E120D6EFDAB5A1261C6020A1C120D52
:10075D002EE0B40215120D2EA3E0B40A0DE55DB422
:10076D000308AF5A12634D020A1C120D2EE0B4029B
:10077D0016120D2EA3E0B4010EE55DB40E09120E96
:10078D00EF122D7A020A1C120D2EE0B40216120D74
:10079D002EA3E0B4020EE55DB40709120EEF12525E
:1007AD00D6020A1C120D2EE0B40215120D2EA3E076
:1007BD00B4090DE55DB40308AF5A125430020A1C9A
:1007CD00120D2EE064027019120D2EA3E0B4091162
:1007DD00E55DB4040C120D2E120F6412672E020A81
:1007ED001C120D2EE064037021120D2EA3E0640A7D
:1007FD007018E55D64057012120D2E120D6EFD124E
:10080D006D8AAD5A124725020A1C120D2EE06403A3
:10081D007029120D2EA3E064017020E55DD39405BF
:10082D004019120D2E120D6EFD126D8A855A62AB96
:10083D005DAD5CAC5B123DFF020A1C120D2EE06437
:10084D00037021120D2EA3E064027018E55D64059E
:10085D007012120D2E120D6EFD126D8AAD5A125FB1
:10086D00A8020A1C120D2EE0B40315120D2EA3E0E2
:10087D00B4030DE55DB40308AF5A126024020A1CDF
:10088D00120D2EE0B40318120D2EA3E0B40410E5E2
:10089D005DD394034009120F4D1249BA020A1C127E
:1008AD000D2EE0B40315120D2EA3E0B4050DE55D7C
:1008BD00B40308AF5A126D78020A1C120D2EE0B463
:1008CD000316120D2EA3E0B4060EE55DB405091254
:1008DD000EEF126868020A1C120D2EE064037019E7
:1008ED00120D2EA3E0B40711E55DB4040C120D2E0C
:1008FD00120F64126B97020A1C120D2EE0B4031630
:10090D00120D2EA3E0B4080EE55DB40409120EEF2E
:10091D0012688D020A1C120D2EE064057014E55D3F
:10092D00B4040F120D24A3A3E0FDAB5A121F7102E4
:10093D000A1C120D2EE0B40516120D72B40B10E543
:10094D005DD394054009120F4D12337D020A1C121E
:10095D000D2EE064067014E55DB4040F120D24A392
:10096D00A3E0FDAB5A122163020A1C120D2EE0B456
:10097D000616120D72B40B10E55DD39405400912E5
:10098D000F4D122694020A1C120D2EE06409701AE6
:10099D00120D2EA3E0B40A12E55DB4040D120D2E56
:1009AD00A3A3E0FF125D94020A1C120D2EE0640950
:1009BD007018120D2EA3E0B40110E55DB4040B12F6
:1009CD000D2E120F641262A98045120D2EE0B4098E
:1009DD0017120D2EA3E0B4020FE55DD39404400869
:1009ED00120EED1214CD8027120D2EE06409701A2F
:1009FD00120D2EA3E0B40310E55DB4040B120D2E01
:100A0D00120F64125D0280078000AF5A126BB42082
:100A1D002A030205A2C21ED22DAF5A1259B97D600A
:100A2D007F0212665F7D327F0312665F7F03126E57
:0F0A3D00DE125DDC7FFF126E9DE47885F6C2232A
:080A4C0022FD126D8AAD5A2251
:08171B008E5E8F5F8D608B6113
:10172300120EDBFFE55F2404120D83FD1264228F8A
:101733006274E22562F562C39400500302191CE54A
:10174300629414400302191CE5616406701D120DB6
:101753007FB4010C120DC7120E947401F002191814
:10176300120DC7120E94E4F0021918E561640E60BD
:101773000302183AE55F240C120D83FFB40A14E543
:101783005F240D120D83B40A0A120DC7120E24E44E
:10179300F08013E55F240D120D83FD126C0B120D07
:1017A300C7120E24EFF0E55F240A120D83FFB40A7B
:1017B30014E55F240B120D83B40A0A120DC7120E2F
:1017C30072E4F08013E55F240B120D83FD126C0BA2
:1017D300120DC7120E72EFF0E55F2409120D83FF9D
:1017E300640A6006EFD39409400A120DC7120E482B
:1017F300E4F08010E55F2409120D83FF120DC71278
:101803000E48EFF0120D7FFFB40B15E55F240612AF
:101813000D83B40B0B120DC7120DFE74FFF080087D
:10182300121948120DFEEFF0121924120DBC120EFC
:10183300947401F0021918E561640A706E120DC701
:10184300120E24E4120DC6120E72E4F0E55F2409B1
:10185300120D83FF640A6006EFD39409400A120D48
:10186300C7120E48E4F08010E55F2409120D83FFD0
:10187300120DC7120E48EFF0120D7FFFB40B15E5E2
:101883005F2406120D83B40B0B120DC7120DFE74E9
:10189300FFF08008121948120DFEEFF012192412FE
:1018A3000DBC120E947401F0021918E561640970FD
:1018B30068120DC7120E24E4120DC6120E72E41242
:1018C3000DC6120E48E4F0120D7FFFB40B15E55F51
:1018D3002406120D83B40B0B120DC7120DFE74FFF9
:1018E300F08013E55F2406120D83FD126C0B120DBD
:1018F300C7120DFEEFF0E55F2407120D83FFE55FCE
:101903002408120D83FD126C0B120DC7120DBC12AD
:101913000E947401F0D22C8002C22CAF60126E734D
:1019230022E55F2407F582E4355EF583E0FFE55F9A
:101933002408F582E4355EF583E0FD126C0BE56265
:1019430075F007A422E55F2406F582E4355EF5838E
:0C195300E0FD126C0BE56275F007A422A9
:103124008F5E8D5FE55ED3941D5003023230E55E01
:1031340094324003023230D22DAF5F1259B97D462A
:103144007F0712665FAF5E1235A474E2255EF55EFA
:10315400120E20E07021120E6CE0701B120E42E081
:103164007015120DF8E0700F120F3C700A123249FC
:103174007D537F02023226123238E55E75F007A4D1
:10318400120E94E070047D3680027D387F0612664C
:103194005F123238120E1EE0FFD394014034EF94D4
:1031A40013502F7D097F0612665F120E1E123240E5
:1031B4007FF47E01126C277D0E7F0312665F7D35DE
:1031C4007F0612665F7D097F0612665F120E6C121F
:1031D40032407FF47E01126C27120E42E0FF60053C
:1031E400125A5C800A1232497D0F7F0312665F7D9A
:1031F400277F0212665F120DF8E0FFF46008126C7C
:10320400C71235A480077D187F0212665F7D377F61
:103214000412665F120F3CFF126CC71235A47D05C1
:103224007F0612665FC22DAF5F0259B9C22CAF5F31
:10323400126E73227FF47E01126C2722E0FF126C5F
:0D324400C71235A4227D187F0212665F229A
:02618C008D5E26
:10618E00EFD3941D402AEF9432502574E22FFFE492
:10619E00FEEEFD3395E0FCEF75F007A42450F5827A
:1061AE00E4340A120E35E4F00EBE07E5D22C80025E
:0761BE00C22CAF5E126E73EC
:0161C50022B7
:062D7A008E5E8F5F8D608C
:102D8000D22B120EDBFFE55F2404120D9D122EA143
:102D9000C39418501C855F82855E83A3A3A3E0FFC4
:102DA000E55F2404120D9DFD126D527883A6078005
:102DB00006E47883F6C22B120D8C122EA1C3943C2C
:102DC000500D120D8CFD126D527884A6078006E41A
:102DD0007884F6C22BE55F2407120D9DFF126E0565
:102DE0008F61E561D394004017E56194085011E5C7
:102DF0005F2407120D9DFF126E057880A6078006DE
:102E000078807601C22BE55F2408120D9DFFE55FF7
:102E10002409120D9D122EAA401FE561942050191D
:102E2000E55F2408120D9DFFE55F2409120D9DFD4D
:102E3000126D527888A607800678887601C22BE545
:102E40005F240A120D9DFFE55F240B120D9D122ECB
:102E5000AA401FE561940D5019E55F240A120D9DEB
:102E6000FFE55F240B120D9DFD126D527881A607C0
:102E7000800678817601C22BE55F240C120D9DFF40
:102E8000E55F240D120D9DFD126D527882A607306C
:102E90002B071257A5D22C8002C22CAF60126E7382
:102EA00022FD1264228F61E56122FD1264228F618E
:062EB000E561D39400224D
:0652D6008E5E8F5F8D600B
:1052DC00D22B120EDBFFE55F2404120E6312534136
:1052EC009418501C855F82855E83A3A3A3E0FFE521
:1052FC005F2404120E63FD126D527883A60780069C
:10530C00E47883F6C22B120E52125341943C500D8A
:10531C00120E52FD126D527884A6078006E4788432
:10532C00F6C22B302B071257A5D22C8002C22CAF01
:04533C0060126E731A
:0B53400022FD1264228F61E561C32290
:106E0500120EBB4008EF6480948A5001227F002255
:106D5200AE05126E05EFC454F0FDAF06126E05EFDC
:036D62004DFF22C0
:10634D008F5ED22D1259B97D1E7F0812665F7D2694
:10635D007F0812665F7D527F0412665FC22B126842
:10636D0042125C6E7880E6FF125A5C125963C22DA0
:06637D00AF5E1259B922C7
:10672E008D5EEFD3940A4006EFD3940F4003EF70C3
:10673E000E90002BEFF0D22CAF5E126E73D322C2EE
:08674E002CAF5E126E73C32232
:025430008F5E8D
:10543200D22D1259B97D207F0512665F7D2E7F0322
:1054420012665F7D527F0412665F90002BE0F55F6B
:10545200E55FB40B067D5F7F078034E55FB40C0621
:105462007D5E7F068029E55FB40D067D0A7F02809E
:105472001EE55FB40E067D327F028013E55FB40F36
:10548200067D467F028008E55F70077D0A7F031272
:09549200665FC22DAF5E1259B92C
:01549B0022EE
:106B97008D5E120EBB400EEF648094865007126321
:0D6BA700EED22C8002C22CAF5E126E732263
:026868008D5E43
:10686A00120EC2126422120EBB4010EF648094A171
:10687A005009900029EFF0D22C8002C22CAF5E1290
:02688A006E732B
:01688C0022E9
:02688D008D5E1E
:10688F00120EC2126422120EBB4010EF648094A14C
:10689F005009900028EFF0D22C8002C22CAF5E126C
:0268AF006E7306
:0168B10022C4
:106D6500D3EF648094814008EF64809489500122B8
:036D75007F00227A
:106E1500120EBB4008EF648094A15001227F00222E
:0814CD008E5E8F5F8D608B6164
:1014D500120EDB14F56374FC2561F5616403600F7E
:1014E500E56164076009E561640B60030216B8C332
:1014F500E5636480948050030216B8E563648094C4
:101505008840030216B8E4F562120D657803C3330B
:10151500CE33CED8F92430F58274003EF583AF6220
:10152500EF3395E0FE120DE0E4F00562E562B408E4
:10153500D8756204E56164037029120D411216FE27
:10154500120D637803C333CE33CED8F9120D36A30B
:10155500A3120D5E7803C333CE33CED8F9120FC56F
:101565000216AFE56164077069120D411216FE128D
:101575000D637803C333CE33CED8F9120D36A3A34A
:10158500120D5E7803C333CE33CED8F9120FC512D0
:101595000D3CA3A3A3120D5E7803C333CE33CED87F
:1015A500F92432F5827400120D3C1216C0C333CEF5
:1015B50033CED8F92433F5827400120D3C120D5345
:1015C5007803C333CE33CED8F92434F582740002C0
:1015D50016AFE561640B60030216B8120D41E01207
:1015E5000EF6A3E0FD126422126E15120D63780348
:1015F500C333CE33CED8F9120D36A3A3120D5E78C0
:1016050003C333CE33CED8F9120FC5120D3CA3A3B5
:10161500A3120D5E7803C333CE33CED8F92432F549
:10162500827400120D3C1216C0C333CE33CED8F9E6
:101635002433F5827400120D3C120D537803C33325
:10164500CE33CED8F92434F5827400120D3CE582F0
:101655002407120D577803C333CE33CED8F924357A
:10166500F5827400120D3CE5822408120E15120E47
:10167500F6E5822409120E15FD126422126E15126A
:101685000D637803C333CE33CED8F92436F582748F
:1016950000120D3CE582240A120D577803C333CEA0
:1016A50033CED8F92437F58274003EF583EDF0D2B8
:0A16B5002C8002C22CAF60126E738D
:1016BF0022E5822404F582E43583F583E0FFE562B9
:1016CF00FD3395E0FCE55F2DF582E55E3CF583E5A6
:1016DF00822405F582E43583F583E0FD126422123E
:1016EF006E15AD07AF63EF3395E0FEEF780322E0A1
:1016FF00FFE562FD3395E0FCE55F2DF582E55E3C8D
:0C170F00F583A3E0FD126422126E152287
:045D02008D5EAC07FF
:105D0600D3EC648094804035EC64809489502EE412
:105D1600FDECFF3395E0FEEF7803C333CE33CED8E8
:105D2600F92428F58274003EF583EDFF3395E0FEF5
:105D3600120DE0E4F00DBD08D8D22C8002C22CAFC3
:045D46005E126E7308
:015D4A002236
:1062A9008D5E120EBB402FEF648094895028EF1445
:1062B900FFE55E24FF922B124FE2D22DAF5E1259F9
:1062C900B97542017F327E00126C27E54270FCC22B
:0762D9002DAF5E1259B9223E
:084670008F5E8C5F8D608B6191
:10467800856082855F83120E08FD1264228F62E5D1
:1046880062D39400500302471DE56294324003024E
:10469800471DE55E64067036D22DAF611259B97DAB
:1046A800527F0512665FAF621235A4120F24B4015F
:1046B8000A120E7C7401F07D388007120E7CE4F03B
:1046C8007D367F0612665FC22DAF610259B9E5607B
:1046D8002406120F28640B703C120F24B401081230
:1046E8000E7C7401F08005120E7CE4F074F9255EEE
:1046F800F55E75F004123984AFF0EF7014E56024AC
:1047080006FBE4355FFAAD62E4FF1234A4D22C80D4
:0C47180006C22C8002C22CAF61126E732E
:014724002272
:082FF0008F5E8C5F8D608B6128
:102FF800856082855F83120E08FD1264228F62E568
:1030080062D39400500302311CE562942840030205
:10301800311CE55E64067037D22DAF611259B97D57
:10302800527F0512665FAF621235A4120EAFE0B48C
:10303800010A120E887401F07D388007120E88E4A8
:10304800F07D367F0612665FC22DAF610259B9E581
:10305800602406120EB3E0640B600302311C120EEA
:10306800AFE0B40108120E887401F08005120E88D2
:10307800E4F0E4FFFEE5602407120EB3E5822E12A9
:103088000E15B40B04AF0680040EBE08E8EF7003FB
:1030980002311CC39408507C120F31EFF07E01EF0F
:1030A8002401FDE433FCEEC39DEC6480F874809841
:1030B8005020E5602406120EB3E5822E120E15FD8F
:1030C800120F31E5822EF582E43583F583EDF00E9B
:1030D80080CDE5602408120EB3E5822F120E156428
:1030E8000B602DEF2408FEC3E55E9EF55E75F004C7
:1030F800123984AEF0EE701CE5602407FDE4355FFC
:10310800FC7E00ED2FFBEE3CFAAD627F011234A489
:0B311800D22C8002C22CAF61126E733B
:013123002289
:0834A4008F638D648A658B665D
:1034AC00756801E4F567120DAAE0FF6409703E121D
:1034BC0035958003120F09D8FB120DA612358778AB
:1034CC0008EF088003120F09D8FB120DA6A3A3E086
:1034DC00FFE568FD3395E0FCE5662DF582E5653C7E
:1034EC00F583A3A3A3E0FD126D8A023540120DAA49
:1034FC00E0FF1235958003120F09D8FB120DA612AE
:10350C0035877804EF088003120F09D8FB120DA63B
:10351C00A3A3E0FF126ED4EF426AAE69AF6A7804DF
:10352C00EF088003120F09D8FB120DA6A3A3A3E08A
:10353C00FF126ED4EF426AE563700FAF67120D672E
:10354C00120EA5E564900AC08012E563B40117AFB2
:10355C0067120D67120EA5E564900530120DDDE5BE
:10356C0069F0A3E56AF074042568F5680567C3E59E
:0A357C00676480949050030234B29B
:1035860022A3E0FF126ED4EF426AAE69AF6A22123E
:0E3596006ED47569008F6AAE697804EF082262
:0A6ED400EFD3940940037F0022224F
:023A70008B5E6B
:103A72001264228F61E561D394005003023B52E548
:103A82006194334003023B52D22DAF5E1259B97D8D
:103A9200527F0512665FAF611235A4746F25611201
:103AA2000E8CE060047D3880027D367F0612665FF0
:103AB2007F2C7E01126C27E561120F33E0F55F70F7
:103AC200077D1B7F0612665F7D577F0212665FE5E8
:103AD2005F603B756001AF5F120D672401FFE43E3A
:103AE200FEAD60ED3395E0FCC3ED9FEE6480F8EC33
:103AF2006480985019120DCEE0B40A04E4FD8006E9
:103B0200120DCEE0FDE4FF12665F056080C87F2CD7
:103B12007E01126C27E561900530120F7F90000044
:103B2200EEF0A3EFF04E70077D1B7F0612665F7DFD
:103B32000C7F0312665F900000E07002A3E0600950
:103B4200E56114FD7F01122ADCC22DAF5E0259B974
:073B5200C22CAF5E126E737E
:013B59002249
:024DBA008B5E0E
:104DBC001264228F5FE55FD394004077E55F9433F4
:104DCC005071D22DAF5E1259B97D527F0512665FBC
:104DDC00AF5F1235A4749F255F120E80E060047DD6
:104DEC003880027D367F0612665F7F2C7E01126C46
:104DFC00277F2C7E01126C27E55F900AC0120F7F73
:104E0C00900000EEF0A3EFF04E70077D1B7F0612B2
:104E1C00665F7D0C7F0312665F900000E07002A35A
:104E2C00E06009E55F14FDE4FF122ADCC22DAF5EE1
:0A4E3C000259B9C22CAF5E126E736A
:014E46002249
:0261C6008B5EEE
:1061C800126422AD07EDD394004025ED943350209E
:1061D800E4FC120E9EED900AC0120DDDE4F0A3F06F
:1061E8000CBC10EE749F2D120E80E4F0D22C8002AD
:0761F800C22CAF5E126E73B2
:0161FF00227D
:025AF7008B5EC4
:105AF900126422AD07EDD394004036ED9433503152
:105B0900E4FC120E9EED900530120DDDE4F0A3F0D9
:105B19000CBC10EE746F2D120E8CE4F0FCECFF330C
:105B290095E0FEED120DD7E4F00CBC08F0D22C8004
:085B390002C22CAF5E126E7374
:015B41002241
:042ADC008F628D6315
:102AE000E4F564E5627052AF64120D6725E0FDEE17
:102AF00033FCAF63120D677805C333CE33CED8F9FC
:102B0000120E2E120F8B8003120F10D8FB120F6BB8
:102B10008003120F10D8FB540FF566AF63120D67D8
:102B20007805C333CE33CED8F9120E2E120F97800C
:102B300003120F10D8FB022B9AE56264017064AF98
:102B400064120D6725E0FDEE33FCAF63120D67786C
:102B500005C333CE33CED8F92450F5827405120E56
:102B600034120F8B8003120F10D8FB120F6B8003EF
:102B7000120F10D8FB540FF566AF63120D6778057E
:102B8000C333CE33CED8F92450F5827405120E34F7
:102B9000120F978003120F10D8FB540FF567ED54F6
:102BA0000FF568E565700CE5667008E5677004E58B
:102BB00068607CAD65E4FF12665FAD66E4FF126697
:102BC0005FE56564097045856769AF69FE7804EF64
:102BD000088003120F09D8FBF569E5684269E569C9
:102BE000B4990B7D09E4FF12665F7D098027E569D2
:102BF00075F00A84F56AFDE4FF12665FE56A75F018
:102C00000AA4FFC3E5699FF56AFD8009AD67E4FF8B
:102C100012665FAD68E4FF12665F7FF47E01126C9E
:0F2C2000270564C3E564648094A05003022AE38F
:012C2F002282
:10642200EFD394004015EF940B5010EFC3940A5031
:1064320008EF75F00AA4FE8002E4FEEDD39400405A
:106442000EED940B5009EDC3940A5003ED2EFEAFEE
:016452000643
:016453002226
:0649BA008E5E8F5F8B6032
:1049C000756105756240D3ED64809484407CED642C
:1049D0008094A55075ED24FDF563D39404406BE5F8
:1049E0006320E06613F5640562E562AE617002055E
:1049F0006114F5828E83E564F07403255FF55FE44E
:104A0000355EF55EE4F563E563C395645033855F19
:104A100082855E83E0FFA3E0FD126D8A0562E56298
:104A2000AC617002056114F5828C83EFF0055FE5DF
:104A30005F7002055E055FE55F7002055E056380DD
:104A4000C6D22CAF60126E73D322C22CAF60126E2E
:024A500073C32E
:014A52002241
:043DFF008C5F8D60E8
:103E0300120EBB5003023ED7EF6480949540030229
:103E13003ED7EB648094875003023ED7EB648094D3
:103E2300E44003023ED7120D677805C333CE33CE89
:103E3300D8F9120FCCF5638F64EB24FBF565D394AB
:103E4300025003023ED7E56575F00384E5F0600395
:103E5300023ED7E56575F00384F567C3941050748B
:103E6300120F787002056314F5828E83E567F07490
:103E730005120FD6E4F565E565C395675052120F39
:103E8300E0E0F566B40A10120F787002056314F5CA
:103E9300828E83E4F0800F120F787002056314F5AD
:103EA300828E83E566F0120FE0A3E0FF120FE0A31A
:103EB300A3E0FD126D8A8F66120F787002056314FA
:103EC300F5828E83E566F07403120FD6056580A72D
:0B3ED300D22C8002C22CAF62126E7372
:013EDE0022C1
:082694008E5E8F5F8D608B618B
:10269C00C22B120FE7600302273112280C500302E1
:1026AC00272CE5649408E56394075074C3E56064D3
:1026BC0080948A506B120EE4A3E0F562B40106908C
:1026CC000520022781E562B40206900522022781CB
:1026DC00E562B40306900524022781E562B4040682
:1026EC00900526022781E562B4050690052802278D
:1026FC0081E562B4060690052A022781E562B407DB
:10270C000690052C022781E562B4080590052E8001
:10271C0064E562B40905900530805AD22B0227FD7E
:10272C00D22B0227FD120EE4E064017052AD60AFB3
:10273C005FAE5E12280C50030227FDE5649408E599
:10274C0063940740030227FDC3E5606480948A40CC
:10275C00030227FD120EE4A3E0F562B40A0590050E
:10276C00328012E562B401059005348008E562B44C
:10277C000209900536E563F0A3806FD22B807212AC
:10278C000EE4E06402706AAD60AF5FAE5E125B4255
:10279C007563008F64C3E5649463E56394005051E2
:1027AC00C3E560648094885048120EE4A3E0F5629F
:1027BC00B40107900538EFF08037E562B40205905C
:1027CC0005398026E562B4030590053A801CE56264
:1027DC00B4040590053B8012E562B4050590053CF8
:1027EC008008E562B4060890053DE564F08002D2ED
:0F27FC002B302B04C22C8002D22CAF61126E73D3
:10280B00221248798E638F64D3E564943BE563941D
:02281B00002299
:064879008E658F66A905A3
:10487F007D057C00120FAFE0C3940A4005120FAF05
:10488F00E4F00DBD00010CED640A4C70E7B90607AA
:10489F00120DEBFF7E0022E964077010120DEB750D
:1048AF00F00AA4ACF0FDE5662406801BE9640870ED
:1048BF0021120DEB75F064A4ACF0FDE56624061231
:1048CF000DEF120F172407120DEF2DFDE43CAF056E
:1048DF00FE22E964097033120DEBFF7E007C037D2D
:1048EF00E81239A6AC06AD07E5662406120DEF7582
:1048FF00F064120F1A2407120DEF120F172408126B
:0D490F000DEF2DFDE43CFEAF0522E4FEFFA0
:01491C002278
:065B42008E658F66A905C7
:105B48007F057E00120FBAE0C3940A4005120FBA0F
:105B5800E4F00FBF00010EEF64084E70E7E9640738
:105B68007020E5662405F582E43565F583E075F077
:105B78000AA4FFE5662406F582E43565F583E02F7F
:045B8800FF227F0079
:015B8C0022F6
:08337D008E5E8F5F8D608B6195
:10338500C22BD3E56064809484500302342BE5603E
:103395006480948D400302342B120FE760030234DE
:1033A5002B120EDB123A4A33CB0133D60233E1033B
:1033B50033EB0433F50533FF0634090734130834BA
:1033C5001D0900003427756201756300D22B023494
:1033D50062756201756308D22B02346275620175EC
:1033E5006310D22B8077756201756318D22B806DBF
:1033F500756201756320D22B806375620175632840
:10340500D22B8059756201756330D22B804F75625E
:1034150001756338D22B8045756201756340D22BE7
:10342500803BC22B8037D3E56064809484402EE5D1
:10343500606480948D5026855F82855E83A3A3E0BA
:10344500B4011A855F82855E83A3A3A3E024F67089
:103455000A756201756358D22B8002C22B302B3757
:10346500E4FF120F56E4F00FBF08F7E56024FB8573
:103475006382856283F07F01E55F2404F582E4358C
:103485005EF583E5822F120E15FE120F56EEF00F34
:0E349500BF08E5D22C8002C22CAF61126E730C
:0134A3002206
:044725008F5E8D5FB7
:10472900E55ED3940050030247C8E55E9415400343
:104739000247C8D22DAF5F1259B97D5F7F05126656
:104749005FAD5EE4FF12665F7D527F0412665F7F94
:10475900F47E01126C2775F020E55E900280123A12
:104769003EAF828583628F63E0F560603DD394003C
:104779004046E56094105040E56025E0F5607561BC
:1047890001E5602401FFE433FEC3E5619FEE648027
:10479900F87480985022120FA3E0FF120FA3A3E030
:1047A900FD1265170561056180D77D1B7F061266BD
:1047B9005F7D5F7F0512665FC22DAF5F0259B9C287
:0647C9002CAF5F126E73BD
:0147CF0022C7
:102163008F5E8D5F8B60E55E640A7074E55FC39478
:102173000A40030222D0122306E4FDFF12665FAD7C
:102183005F1222DFE55F123A4A21AB0121B102213E
:10219300B70321BD0421C30521C90621CF0721D5DA
:1021A3000821DB09000021E090052002222A900586
:1021B3002202222A90052402222A90052602222A9C
:1021C30090052802222A90052A02222A90052C0231
:1021D300222A90052E02222A900530804A0222C923
:1021E300E55E64017052E55FD394004006E55F94B9
:1021F300034006E55F640A703C122306E55FB40AF8
:102203000A7D0A1222DF900532801CE55FB4010AC1
:102213007D0B1222EC900534800DE55FB402137D33
:102223000C1222EC900536E0FEA3E0FF1264860256
:1022330022D70222C90222D0E55E64026003022291
:10224300D7E55FD3940050030222D0E55F94075093
:102253007CD22DAF601259B97D277F0812665F7D4E
:1022630006E4FF12665F7D14E4FF12665FE55F24F8
:10227300FE601A14602114602814602F1460362441
:102283000570437D011222F990053880307D0212DA
:1022930022F990053980267D0312231C90053A808C
:1022A3001C7D0412231C90053B80127D05122329FB
:1022B30090053C80087D0612232990053DE0FF7EB2
:1022C300001264B7800EAF60126BB48007C22CAFEC
:1022D30060126E73C22DAF601259B922E4FF126609
:1022E3005F7D527F0412665F22E4FF12665F7D52B8
:1022F3007F0412665F22E4FF12665F7D527F041241
:10230300665F22D22DAF601259B97D277F0812660E
:102313005F7D06E4FF12665F22E4FF12665F7D5273
:102323007F0412665F22E4FF12665F7D527F041210
:03233300665F22C0
:044AEB008E638F64E3
:104AEF000564E5647002056314F5828E83E0F56654
:104AFF00607AC3940850757F2C7E01126C27E4F501
:104B0F0065E565C395665064856482856383E012AD
:104B1F003A4A4B5C004B3A0A4B3E0B4B440C4B4A08
:104B2F000D4B500E4B560F00004B62E4FD802D7D58
:104B3F005F7F0780287D5E7F0680227D0A7F02804F
:104B4F001C7D327F0280167D467F0280107D0A7F9A
:104B5F0003800A856482856383E0FDE4FF12665F4C
:0C4B6F000564E56470020563056580952F
:014B7B002217
:061F71008F5E8D5F8B60A6
:101F7700C22BE55E640A6003022065E55F123A4AF8
:101F87001FA6011FB9021FCC031FDF041FF2052084
:101F97000806201E07203408204909000020611286
:101FA700209A7D011220E8756101756200D22B022B
:101FB700208112209A7D021220E87561017562085E
:101FC700D22B0220811220B67D031220F575610104
:101FD700756210D22B0220811220B67D041220F5E3
:101FE700756101756218D22B0220811220D212214D
:101FF700487D05122118756101756220D22B0220D8
:10200700811220D21221487D0612211875610175AF
:102017006228D22B02208112210212215C7D071235
:102027002125756101756230D22B022081122102B0
:1020370012215C7D08122125756101756238D22B4A
:102047008038122132E4FDFF12665F7D0912214FAD
:10205700756101756240D22B8020C22B801CE55E22
:1020670064017016E55F24F670101221327D0A12A2
:10207700214F756101756258D22B302B09AF62AEC3
:1020870061124AEB8005AF60126BB4C22DAF6012CC
:0220970059B935
:1020990022D22DAF601259B97D577F0212665F7D3A
:1020A90005E4FF12665FE4FDFF12665F22D22DAFE1
:1020B900601259B97D577F0212665F7D05E4FF12F0
:1020C900665FE4FDFF12665F22D22DAF601259B937
:1020D9007D577F0212665F7D05E4FF12665F22E489
:1020E900FF12665F7D527F0412665F22E4FF12666B
:1020F9005F7D527F0412665F22D22DAF601259B9FB
:102109007D577F0212665F7D05E4FF12665F22E458
:10211900FF12665F7D527F0412665F22E4FF12663A
:102129005F7D527F0412665F22D22DAF601259B9CA
:102139007D577F0212665F7D05E4FF12665F22E428
:10214900FDFF12665F22E4FF12665F7D527F041273
:0A215900665F22E4FDFF12665F22BC
:1035A4008F72E572D3945940107D5A12368B24A63B
:1035B400FD700302368A023685E572D3944F4016B5
:1035C400E572945A50107D5012368B24B0FD70036E
:1035D40002368A023685E572D394454016E5729424
:1035E4005050107D4612369324BAFD700302368A79
:1035F400023685E572D3943B4012E5729446500C32
:103604007D3C12369324C4FD607C8075E572D394AE
:10361400314012E572943C500C7D3212369B24CE1C
:10362400FD6063805CE572D394274012E5729432A6
:10363400500C7D2812369B24D8FD604A8043E572E5
:10364400D3941D4016E572942850107D1EE4FF1299
:10365400665FE57224E2FD602D8026E572D3941343
:103664004016E572941E50107D14E4FF12665FE567
:103674007224ECFD60108009E572C394145007AD08
:1036840072E4FF12665F22E4FF12665FE57222E4D1
:0F369400FF12665FE57222E4FF12665FE57222A5
:1059B9008F6AE56A700C302D097F01126EF17FC084
:1059C900801FE56A700C202D097F01126EDE7FC0F1
:1059D9008026E56AB40112302D0F7F02126EF17F25
:1059E90030120016C22F026969E56AB40114202D2C
:1059F900117F02126EDE7F30126E9D7FC87E00120B
:035A09006C2722E5
:106945008F69D22D1259B97D607F0212665F7D3243
:106955007F0612665F7D1E7F0512665FC22DAF69D9
:046965001259B922E8
:106BB4008F69D22D1259B97D607F0212665F7D30D4
:0D6BC4007F0312665FC22DAF691259B9221E
:0E6E73008F68302C03026945AF68126BB422A1
:105D9400EF24FE60101460162402701C7F01126E42
:105DA400F17F8080107F02126EF17F2080077F03D5
:105DB400126EF17FA01200167FF47E01126C27751B
:105DC4004204E54270FC7F647E00126C277F03125C
:085DD4006EDE7FA0126E9D221D
:1064B7008E618F627C007D0A1239B8AD07E4FF1246
:1064C700665F7D5B7F0612665FAE61AF627C007DB3
:1064D7000A1239B8E4FF12665F7D4A7F0702665FDA
:046486008E618F6232
:10648A007C007D3C1239B81235A47D057F06126660
:10649A005FAE61AF627C007D3C1239B8ED4C600C96
:0C64AA00AF051235A47D4A7F0712665F23
:0164B60022C3
:025FA8008D5E0C
:105FAA00120EBB402FEF648094955028120D67782B
:105FBA0005C333CE33CED8F9120FCCFEE4FD0FEF72
:105FCA00AA0670010E14F5828A83E4F00DBD20EE54
:0B5FDA00D22C8002C22CAF5E126E734E
:015FE5002299
:106024008F5E900540E0D394024015D22D1259B9E9
:106034007542037F327E00126C27E54270FC8015A6
:10604400D22DAF5E1259B97D1B7F0612665F7D0C9F
:0D6054007F0312665FC22DAF5E1259B922A4
:106D78007E10900540E4F0A3DEFC7E10D22C126E4B
:016D88007397
:016D890022E7
:106D8A00BF0A02E4FFBD0A02E4FDEF75F00AA42D72
:026D9A00FF22D6
:106C0B00EFD394094002E4FFEDD394094002E4FD75
:0C6C1B007804EF08800123D8FD4DFF2213
:1040860007010203040506070707060504030201E4
:1040960003010A0A030307050303020503020A0ACA
:1040A60004050A0A0104050A0A0A04050A0A0203A3
:1040B600070A0A03040A0A04024B00020032072E0A
:1040C60003024B0002003202055F000302055F0097
:1040D6000402055F000502055F000604072E082698
:1040E6000640033204072E08260640025304081E23
:1040F60008260452010008024B00020032072E086F
:104106001E08260452010003072B02350636030754
:104116002B0235063803072B0235072603072B0229
:1041260035025302055F000F02055F001002055FAE
:10413600001102055F001202055F001302055F0011
:0A41460014080C0A1D020500241BDA
:10525D007461F0A37420F0A37452F0A37401F0A351
:10526D0022A3F0A37461F0A37440F022F0A37403A1
:10527D00F0E4A3F0A37410F0A37403F0E4A3F0A37F
:10528D00227461F0A37441F0A3227461F0A3F0A322
:10529D007430F0A3227496F0A37432F0A37495F0D9
:1052AD00A3741EF0A322F0A37461F0A314F0A374F1
:1052BD0070F0A3E4F022A3F0A37452F0A3223CF506
:0952CD0083E0FEEF3395E0FC22C2
:10003E007E407F867C017D507B08125EA67E407FCF
:10004E008E7C017D587B08125EA67E407F967C01D9
:10005E007D007B04125EA67E407FA27C017D087B24
:10006E0004125EA67E407F9E7C017D107B04125E94
:10007E00A67E407F9A7C017D187B04125EA67E4090
:10008E007FAB7C017D207B05125EA67E407FA67C29
:10009E00017D287B05125EA67E407FB07C017D30FF
:1000AE007B05125EA67E407FB57C017D387B0412F7
:1000BE005EA67E407FB97C017D407B04125EA67EEB
:1000CE00407FBD7C027DA07B09125EA67E407FC66E
:1000DE007C027DC07B07125EA67E407FCD7C027DBA
:1000EE00E07B05125EA67E407FD27C037D007B0501
:1000FE00125EA67E407FD77C037D207B05125EA616
:10010E007E407FDC7C037D407B05125EA67E407FB9
:10011E00E17C037D607B09125EA67E407FEA7C0354
:10012E007D807B09125EA67E407FF37C037DA07BE3
:10013E0009125EA67E407FFC7C037DC07B11125EA1
:10014E00A67E417F0D7C037DE07B07125EA67E417D
:10015E007F147C047D007B07125EA67E417F1B7C94
:10016E00047D207B07125EA67E417F227C047D40AB
:10017E007B07125EA67E417F297C047D607B051283
:10018E005EA67E417F2E7C047D807B05125EA67E60
:10019E00417F337C047DA07B05125EA67E417F38B5
:1001AE007C047DC07B05125EA67E417F3D7C047D76
:1001BE00E07B05125EA67E417F427C057D007B05BD
:1001CE00125EA67E417F477C057D407B09125EA6AE
:1001DE009000297417F07F031263EE9000287419B3
:1001EE00F090002074B1F09000217491F0900022F4
:1001FE007403F0900023747FF090002404F09000BC
:10020E00257403F0E4900026F0900027F090003063
:10021E0074091252797415F0A37403F0A3741512B5
:10022E0052797409F0A37403F0E4FFEFFD3395E007
:10023E00FC74302DF58274001252CB74102DF582A1
:10024E0074003CF583EEF00FBF08E0E4FFEFFD33E2
:10025E0095E0FC74382DF58274001252CB74182D73
:10026E00F58274003CF583EEF00FBF08E090052098
:10027E00E4F0A374B4F0900522E4F0A374B4F0900B
:10028E0005247401F0A374E0F0900526E4F0A37445
:10029E0078F09005287402F0A37458F090052AE4C3
:1002AE00F0A3743CF090052C7402F0A37458F07413
:1002BE000790052EF0A3F0900530F0A3F0900532D4
:1002CE00F0A3F0900534F0A3F0900536E4F0A3749B
:1002DE003CF0900538740AF09005397428F09005BA
:1002EE003A7405F090053B740AF090053CF09005C9
:1002FE003D7428F09000A47401F0900B607415F01A
:10030E00A37411F09000A57401F0900B807415F099
:10031E00A37410F09000A67401F0900BA07415F069
:10032E00A37421F09000A77401F0900BC07415F027
:10033E00A37420F09000A87401F0900BE07415F0F7
:10034E00A37431F09000A97401F0900C007415F0B4
:10035E00A37430F09000AA7401F0900C207415F084
:10036E00A37441F09000AB7401F0900C407415F042
:10037E00A37440F09000AC7401F0900C60745312B2
:10038E00526774361252677438F0A3E4F0A37453B4
:10039E00F0A3E4F09000AD04F0900C807453125270
:1003AE00677434F0A37421F0A37453F0A3E4F090B7
:1003BE0000AF04F0900CC01252657430F07403124A
:1003CE0052C3E4F09000B004F0900CE01252657449
:1003DE0030F074041252C3E4F09000B104F0900DAA
:1003EE000012525D74321252677452F0A37420F0F0
:1003FE009000B27401F0900D2012525D7432F0A391
:10040E0074021252C47420F09000B37401F0900D77
:10041E004074531252677433F0A3E4F09000B404A6
:10042E00F0900D6012528E7430F0740212526E9073
:10043E0000B57401F0900D8012528E7430F0740578
:10044E0012526E9000B67401F0900DA012528E747E
:10045E0030F0A3740612526F9000B77401F0900D35
:10046E00C012528E1252A27498F0A3744B12526F95
:10047E009000B87401F0900DE012528E1252A274D8
:10048E0093F0A3741812526F9000B97401F0900E8D
:10049E000012528E7430F0A3741312526FA3747044
:1004AE00F0A37402F09000BA14F0900E201252973E
:1004BE007412F0A374701252677461F0A314F0906A
:1004CE0000BB7401F0900E4012529774111252B389
:1004DE009000BC04F07461900E6012529974141264
:1004EE0052B39000D104F090110012528E7492F01B
:1004FE00A3744BF0A37490F0A37402F0A37490F065
:10050E00A37432F07499A3F0A3F0A374601252672F
:10051E0074911252677491F0A3E412526F90000F0F
:10052E007401F0125DDC7F01126EF17F4012001635
:10053E007D2F7F0712665F7D0C7F0312665F7D3213
:0C054E007F0612665F7D1E7F0512665F4F
:01055A00227E
:0A5EA6008E5A8F5B8C5C8D5D8B5E65
:105EB000E4F9C3E55E6480F8E96480985028E9FF5E
:105EC0003395E0FEE55B2FF582E55A3EF583E493DA
:105ED000FFE9FD3395E0FCE55D2DF582E55C3CF5E1
:065EE00083EFF00980CC05
:015EE6002299
:10556B00AF6AEF3395E0FEE56975F008A42428F5E2
:10557B0082E43400F583E5822FF582E5833EF583E3
:10558B00E0FFE56AFD3395E0FC22AB66AD65AF64E9
:10559B00223EF583E0FD74B82FF582741D3EF58332
:1055AB00EDF0056AE56A22EF3395E0FEEF25E0FFAB
:1055BB00EE33FE22A2E0CE13CE13223CF583EFF0A6
:0555CB00056AE56A22FB
:045B8D008C5B8D5C44
:105B9100EF6043D201D202D20CE4F55D855C8285CF
:105BA1005B83E0FEA3E04E6027AF5D1255B2E55C7A
:105BB1002FF582E55B3EF583E0FEA3E0FF1245038E
:105BC100922920290B055DC3E55D6480949040CC4A
:065BD100C201C202C20C79
:015BD70022AB
:045BD8008C608D61EF
:105BDC00EF6043D201D202D20CE4F562856182857A
:105BEC006083E0FEA3E04E6027AF621255B2E56120
:105BFC002FF582E5603EF583E0FEA3E0FF1245033E
:105C0C00922D202D0B0562C3E5626480949040CCEC
:065C1C00C201C202C20C2D
:015C2200225F
:04450300AD07AC064E
:10450700C22E780CEF0880031255BFD8FB540FF565
:10451700637808AF05AE04EF0880031255BFD8FBD8
:10452700540FF5647804AF05AE04EF088003125505
:10453700BFD8FB540FF565ED540FF566E563607161
:10454700B40108125595123C3D8066E563B4020834
:10455700125595126B1F8059E563B40308125595E0
:10456700123896804CE563B40408125595126AC058
:10457700803FE563B405081255951224E68032E5BD
:1045870063B4060812559512125F8025E563B407D8
:1045970008125595125AAB8018E563B408081255EE
:1045A7009512574A800BE563B409061255951268B0
:0345B700B2A22E7F
:0145BA0022DE
:103C3D008F678D688B69E567B40113900020E0FFF5
:103C4D001258B3900020EFF0FD7F20023CFAE5679B
:103C5D00B40211900021123D00900021EFF0FD7F84
:103C6D0021023CFAE567B40311900022123D009049
:103C7D000022EFF0FD7F22023CFAE567B4041090BC
:103C8D000023123D0A900023EFF0FD7F23805EE5B7
:103C9D0067B40516900024123D0A900024EFF0FD44
:103CAD007F247E001263830264E7E567B4061090FB
:103CBD000025123D14900025EFF0FD7F25802EE5A7
:103CCD0067B40710900026123D14900026EFF0FD0A
:103CDD007F268019E567B40819900027E0FFAB69CE
:103CED00AD681258B3900027EFF0FD7F277E0012CC
:103CFD00638322E0FFAB69AD681258B322E0FFABDE
:103D0D0069AD681258B322E0FFAB69AD681258B3C4
:013D1D002283
:1058B300D22FAC07BD01047E018033BD02047E02FA
:1058C300802CBD03047E048025BD04047E08801E55
:1058D300BD05047E108017BD06047E208010BD0721
:1058E300047E408009BD08047E808002C22FBB0174
:1058F30005EE4204800BEB7006EEF452048002C204
:075903002F302F03AF042237
:01590A00227A
:026B1F008B6782
:106B2100C22FEF7016ED7013E5677003025C6EE51E
:0B6B310067B401077880E6FF125A5C91
:016B3C002236
:063896008F678D688B694D
:10389C00E567700712397CE4FD801AE567B401070F
:1038AC0012397C7D01800EE567B4020CAD69AF68FE
:1038BC00126E817D02024F5AE567B40306124D2B3E
:1038CC00C21E22E567B40415AD69AF681264228F7D
:1038DC0043754205E542700302397B80F7E5676466
:1038EC00067017E5687013F56A12556B74102DF598
:1038FC008274001255C6B408F022E567640770178D
:10390C00E5687013F56A12556B74182DF582740006
:10391C001255C6B408F022E56764087027E5687094
:10392C0023E569701FF56AAF6AEF3395E0FE7410FA
:10393C002FF582740012559CB408EC754201E542D7
:10394C00602D80FAE56764097025E5687021E569EA
:10395C00701DF56AAF6AEF3395E0FE74182FF5828F
:0F396C00740012559CB408EC754201E54270FCE2
:09397B0022AD69AF68126E8122D1
:106AC0008F67AE03AF05E567D394004012E5679486
:106AD00007500CAD06126E81AD07AF671266B32288
:1024E6008F678D688B69E5677018E5687014E56914
:1024F60070057F01126E9DE56964016003022693F3
:102506008043E567701CE568B40117E56970057FCF
:1025160004126E9DE569640160030226937F04023E
:102526002690E5677029E56864027023E569700501
:102536007F05126E9DE56964016003022693900093
:102546000FE0B403057F010226907F05022690E581
:1025560067B4011BE5687017E56970057F02126EA6
:102566009DE569640160030226937F02022690E5D9
:1025760067B4011CE568B40117E56970057F0812A8
:102586006E9DE569640160030226937F080226902A
:10259600E56764017029E56864027023E5697005E2
:1025A6007F0A126E9DE5696401600302269390001E
:1025B6000FE0B403057F020226907F0A022690E50B
:1025C60067B4021BE5687017E56970057F40126EF7
:1025D6009DE569640160030226937F40022690E52B
:1025E60067B4021CE568B40117E56970057F10122F
:1025F6006E9DE569640160030226937F10022690B2
:10260600E56764027024E5686402701EE56970057A
:102616007F50126E9DE5696401707290000FE0B400
:1026260003047F4080647F508060E567B40317E54C
:10263600687013E56970057F80126E9DE569640117
:10264600704B7F808044E567B40318E568B40113D6
:10265600E56970057F20126E9DE5696401702E7F25
:10266600208027E56764037024E5686402701EE530
:102676006970057FA0126E9DE569B4011090000F88
:0E268600E0B403047F8080027FA012001622C1
:10125F008F678D688B69E5677017AD69AF68126E20
:10126F00818E348F35D3E5359400E534940050F5F5
:10127F0022E567B4011BE568B40116E5697007C282
:10128F00307F01122EB6E569640160030214CC8031
:10129F0058E5676401702BE56864027025E5697095
:1012AF0007C2307F02122EB6E56964016003021493
:1012BF00CC90000FE0640370030214CCD2307F0295
:1012CF008031E5676401702EE56864037028E56975
:1012DF007007C2307F03122EB6E569640160030206
:1012EF0014CC90000FE0B40306D2307F018004D2FB
:1012FF00307F03022EB6E5676401702DE568640444
:10130F007027E569700CC2307F01122EB67F401234
:10131F006E9DE569640160030214CCD2307F011227
:10132F002EB67F40120016807CE5676401703AE5A7
:10133F006864057034E569700CC2307F02122EB6F6
:10134F007F10126E9DE569640160030214CC90005A
:10135F000FE0640370030214CCD2307F02122EB65A
:10136F007F10120016D22F803EE5676401703BE5B7
:10137F006864067035E569700CC2307F03122EB6B3
:10138F007F50126E9DE569640160030214CCD23068
:10139F007F03122EB690000FE0B403047F4080024B
:1013AF007F50120016C22F026969E5676402702927
:1013BF00E56864017023E56970057F100214B3E5D9
:1013CF0069B401057F100214BDE569640260030270
:1013DF0014CCD22F7F010214C9E56764027029E58E
:1013EF006864027023E56970057F200214B3E56914
:1013FF00B401057F200214BDE56964026003021485
:10140F00CCD22F7F020214C9E56764027029E56808
:10141F0064037023E56970057F400214B3E569B476
:10142F0001057F400214BDE569640260030214CC1C
:10143F00D22F7F030214C9E56764027023E5686445
:10144F0004701DE56970047F808059E569B401045B
:10145F007F80805AE56964027063D22F7F04805ABF
:10146F00E56764027023E5686405701DE569700423
:10147F007F048030E569B401047F048031E569643D
:10148F0002703AD22F7F058031E5676402702EE536
:10149F0068640670287D017F07124ED2401FE569F0
:1014AF0070057F08026EDEE569B401057F08026EE4
:0E14BF00F1E569B40207D22F7F0612297E22C2
:025AAB008B6707
:105AAD00EF7037ED7034E567700690000F048020BD
:105ABD00E567B4010A90000F7402F0D22F801BE548
:105ACD0067B40216C21E7FFF126E9D90000F740305
:105ADD00F0C2307F02122EB6D22F302F0C90000F55
:095AED00E0FD7F0F7E00126383CF
:015AF600228D
:10574A008F678D688B69E567700C12578E749F2F6F
:10575A00F58274008019E567B4010C12578E749FA4
:10576A002FF58274008016E567B402091257963E37
:10577A00F583E4F022E567B403091257963EF583F0
:10578A007401F022AD69AF68126E8122AD69AF680B
:0B579A00126E81746F2FF582740022E4
:0268B2008F67EE
:1068B400AF057804EF08800123D8FD4BF568E56740
:1068C400B40908E568B499030253C0AD68AF671210
:0268D400651746
:0168D600229F
:0D6E8100EF75F00AA47C002DFFEC35F0FE4B
:016E8E0022E1
:0466B3008F688D69F6
:1066B700C3E569648094E4501BE4F56AC3E5696443
:1066C70080F8E56A648098500BC22FAF6812297E64
:0466D700056A80E8E8
:0166DB00229C
:0D6E8F00C296007F0512681C126454D29652
:016E9C0022D3
:106D2600126E8FEF20E0F9C296007F0612681CC231
:066D3600B60000D2962217
:106D3C00126E8FEF20E0F9C296007F0412681CC21D
:066D4C00B60000D2962201
:045FE6008E608F61D9
:105FEA00AE04AF058E638F64C296007F0312681CED
:105FFA00E560FF12681CAF6112681CE4F562126466
:10600A0054E5642562F582E43563F583EFF00562B1
:09601A00E562C3942040E7D29630
:01602300225A
:085C23008E658F668C678D68A9
:105C2B00126E8FEF20E0F985656A85666BC2960070
:105C3B007F0212681CE567FF12681CAF6812681CB4
:105C4B00E4F569E56B2569F582E4356AF583E0FFD8
:105C5B0012681C0569E569C3942040E7C2B60000D1
:025C6B00D296CF
:015C6D002214
:0A5505008E5A8F5B8C5C8D5D8B5E0F
:10550F00C2AF126D26126E8FEF20E0F9855C6085B9
:10551F005D61C296007F0212681CE55AFF12681C7B
:10552F00AF5B12681CE4F55FAF5EEF3395E0FEC32F
:10553F00E55F9FEE6480F87480985014E561255FF5
:10554F00F582E43560F583E0FF12681C055F80D8B3
:0B555F00C2B60000D296126D3CD2AF25
:01556A00221E
:106383008E718F728D73C2AF126D26126E8FEF20D6
:10639300E0F9C296007F0212681CE571FF12681CC7
:1063A300AF7212681CAF7312681CC2B60000D2969B
:0663B300126D3CD2AF2286
:10609E00C2AFE4F55BF55CF55DF55EF55FF55AAE06
:1060AE005EAF5FAC5BAD5C125FE67420255CF55CA9
:1060BE00E4355BF55B7420255FF55FE4355EF55ED8
:0B60CE00055AE55AC3948940D6D2AFB2
:0160D90022A4
:105DDC00C2AF756200756300756400E4F560F5612F
:105DEC00F55F126D26AE63AF64AC60AD61125C23DF
:105DFC0074202561F561E43560F56074202564F547
:105E0C0064E43563F563055FE55FC3948940D312A1
:045E1C006D3CD2AF58
:015E2000225F
:105632000500050105030507050F051F051E051CCD
:10564200051805100201040E040A03060101040BE9
:105652000304040F020304010302040D0200020208
:1056620003000409040403050307010003030407FC
:10567200030104060402040C0516051500000615B4
:0E568200062A060C06380633061E0612061708
:104C9C002430F58274003EF583EDFF3395E0FEE59C
:104CAC00822FF582E5833EF583E0FFEDFB3395E043
:104CBC00FA22AF4112681CC293126EE8D293D2AFA3
:104CCC00223EF583E0FC74B82FF582741D3EF5830B
:104CDC00ECF00D221528E528D394002225E024328F
:104CEC00F582E43456F583E49322E4F57CD20EC2CB
:104CFC0027C21DC21A227FA0126E9DE4F542C21E6D
:104D0C0022126EE8D2B67801EF0822122C30D2CAE9
:0F4D1C00D20ED22722ECFF3395E0FEEF78032270
:10415000200E2F900540E004F577D36480948150C1
:1041600003024210D3E5776480948F400375770F84
:10417000900029E0FF122C3090002AE0F576124CD6
:10418000F622301A58302712124CE0400302421037
:10419000C2CAC227D21D85762822301D0A124CE0E1
:1041A000506EC227C21D22AF7A157AEF700BC21A69
:1041B000E57625E0F528D21D22E57B30E005857601
:1041C000288008E57675F003A4F528AF7B7801EF29
:1041D00008800103D8FDF57BD227D2CA22D5770803
:1041E000C20EE4F542C21E22057C7440257CF58295
:1041F000E43405F583E0124CE8540FF57A7401932A
:10420000F57B700AD21DE57625E025E0F528D21A67
:01421000228B
:1050EB00200E12900029E0FF122C3090002AE0F5E0
:1050FB0078124CF622301A5130270F124CE0505DCB
:10510B00C2CAC227D21D85782822301D0A124CE054
:10511B00504BC227C21D22AF7A157AEF7007C21A05
:10512B00C20EF54222E57B30E0058578288008E544
:10513B007875F003A4F528AF7B7801EF08800103A5
:10514B00D8FDF57BD227D2CA22E543124CE8FA747C
:0D515B000193FBEA540FF57AEBF57BD21AB5
:015168002224
:10645400E4F575D297F574C2B6126EE8AF7578019B
:10646400EF08800123D8FDF57530970343750112B9
:106474006EE8D2B60574C3E5746480948840D8AFDE
:0164840075A2
:0164850022F4
:096EE8000000000000000000227F
:10663300C2B7E4FEC2B6126EE8EF30E704D2B5800B
:1066430002C2B5124D0D800123D8FDFF126EE80E74
:0B665300BE08E1C2B6D2B7D2B6D2B585
:01665E002219
:0D001600C2AFEF4227AF27126633D2AF22F0
:0E6E9D00C2AFEFF45227AF27126633D2AF22F6
:10681C00E4FEC2B6126EE8EF30E704D2B58002C2D5
:10682C00B5124D0D800123D8FDFF126EE80EBE0887
:05683C00E1D2B6D2B567
:016841002234
:096EF100C2AFEF4241124CBE2277
:0A6EDE00C2AFEFF45241124CBE2285
:102C3000EF123A4A2C98012C9F022CA6032CAD04CB
:102C40002CB4052CBB062CC2072CC9082CD0092C8F
:102C5000D70A2CDE0B2CE50C2CEC0D2CF30E2CFAE9
:102C60000F2D01102D08112D0F122D16132D1D14CF
:102C70002D24152D2B162D32172D39182D40192DD9
:102C8000471A2D4E1B2D551C2D571D2D5E1E2D65D3
:102C90001F2D6C2000002D5575CB8E75CAC6227570
:102CA000CB9575CA772275CB9B75CA692275CBA067
:102CB00075CABA2275CBA675CA332275CBAB75CA55
:102CC000632275CBB075CA022275CBB475CAA32234
:102CD00075CBB875CAFA2275CBBC75CAD82275CB2C
:102CE000C075CAA82275CBC475CA362275CBC77504
:102CF000CA862275CBCA75CABC2275CBCD75CAB43B
:102D00002275CBD075CA762275CBD375CA302275A1
:102D1000CBD575CAB22275CBD875CA132275CBDA5A
:102D200075CA522275CBDC75CA7D2275CBDD75CA9A
:102D30006E2275CBE075CA542275CBE275CA1B2290
:102D400075CBE375CAC32275CBE575CA5E2275CB18
:102D5000E675CADA22801C75CBE875CA902275CB5D
:102D6000EA75CAD92275CBEC75CA092275CBED7507
:0A2D7000CA292275CBE875CA41227A
:10002600C3EF648094A15008EF25E025E0F528226F
:04003600E4F52822A3
:02379F008F5A3F
:1037A100900118E0FFE55A7006E545D39F5012E5F8
:1037B1005A64016003023895E546D39F50030238ED
:1037C10095E55A7018C3E5459FF55D74602FF58244
:1037D100E4341EAD82F55E8D5F7F40801BE55AB4F7
:1037E1000119C3E5469FF55D74B02FF582E4341EDF
:1037F100AF82F55E8F5F7F101200167FF47E01129B
:103801006C277D207F0512665F7D1A7F0812665F37
:103811007FC87E00126C27E4F55BE55BC3955D50C4
:1038210061055FE55FAE5E7002055E14F5828E8311
:10383100E0F55C123A4A38720038500A38540B38B5
:103841005A0C38600D38660E386C0F00003878E479
:10385100FD80277D5F7F0780227D5E7F06801C7D46
:103861000A7F0280167D327F0280107D467F0280B2
:103871000A7D0A7F038004AD5CE4FF12665F055B8D
:103881008098E55A70047F408007E55AB401057FAE
:0438910010126E9D06
:013895002210
:10506800200E10754406901DB8E06003D20E22E4AD
:10507800F54222E528D394004003152822C2CA1518
:1050880044E54414603D14603214601D1460151426
:105098007049901DB8E0FF7003F54222122C309041
:1050A8001DB9802F901DBA8015901DBBE0FF7003BD
:1050B800F54222122C30901DBC8018901DBDE0FFD7
:1050C800020026901DBEE0FF7003F54222122C302C
:1050D800901DBFE0FF120026D2CA22E4F542C2CAE0
:0350E800C20E22D3
:10660500900028E0FF6026200E07124D177528140C
:1066150022E528D394004003152822202708D2CA52
:0E662500752814D22722C2CA75287DC22722EA
:1065A700200E0C7F1C124D1775286475793C22E567
:1065B70028D394004003152822AF791579D3EF64C7
:0E65C700809480400475286422C20EE4F542E0
:0165D50022A3
:1062E000E54214601C14601C14601F1460221460CA
:1062F0002224057021C2CAC20EC227C21DE4F54481
:1063000022025068126605D21E22124150D21E226D
:076310000265A71250EB2209
:1063EE00BF010790002A7418F022BF020790002AFE
:1063FE007412F022BF030590002A8014BF04079088
:10640E00002A740BF02290002ABF05047409F022B2
:04641E00740CF022E8
:024FE200AC071A
:104FE400C3EC64809480404AEC64809488504320ED
:104FF4002B21E4FD124D21C333CE33CED8F9124C0C
:105004009C74102BF58274003AF583EFF00DBD0803
:10501400E3801FE4FD124D21C333CE33CED8F91201
:105024004C9C74182BF58274003AF583EFF00DBD97
:1050340008E3202B16E4FDEDFF3395E0FE74102FFA
:10504400F5827400124CCDBD08ED22302B15E4FD21
:10505400EDFF3395E0FE74182FF5827400124CCDE9
:03506400BD08ED97
:015067002226
:1053C0007D3F7F0912665F7D507F0812665F906F98
:1053D0001A1254277D5B7F0612665F906F1B125472
:1053E00027906F1CE493FDE4FF12665F906F1DE44D
:1053F0009324BE601414601514601814601B1460AC
:105400001E240570217D0A80067D3280027D467F44
:105410000280107D0A7F03800A7D287F0380047D3F
:10542000467F0312665F22E493FDE4FF12665F226B
:105F28008F5BE55B7005D22DFF8009E55BB4010747
:105F3800D22D7F011259B97D4B7F0212665F7D0217
:105F4800E4FF12665F7D32E4FF12665F1253C0E51C
:105F58005B70028005E55BB401057F40126E9D22EF
:103D1E00A209300501B350307D017F04124ED250FE
:103D2E002320050E30090B9000A4E0FF7C0B7D6074
:103D3E00800F30050F20090C9000A5E0FF7C0B7D55
:103D4E0080125BD8A2099205A20A300601B3503048
:103D5E007D027F04124ED2502320060E300A0B90A5
:103D6E0000A6E0FF7C0B7DA0800F30060F200A0C12
:103D7E009000A7E0FF7C0B7DC0125BD8A20A9206D2
:103D8E00A20B300701B350307D037F04124ED25088
:103D9E002320070E300B0B9000A8E0FF7C0B7DE07C
:103DAE00800F30070F200B0C9000A9E0FF7C0C7DDC
:103DBE0000125BD8A20B9207A20D300801B350304F
:103DCE007D047F04124ED2502320080E300D0B902E
:103DDE0000AAE0FF7C0C7D20800F30080F200D0C18
:103DEE009000ABE0FF7C0C7D40125BD8A20D9208D8
:013DFE0022A2
:1064E700534103900024E0FE543FFF7804088001E5
:1064F70023D8FD54F0FFEE30E40343070490002453
:0F650700E030E503430708EF4241C2AF124CBE3C
:016516002262
:02297E008F6B5D
:10298000302F05756CF48003756C64E56B64017021
:1029900029AF417803EF08800123D8FD3392307FBF
:1029A0001020300B122A9A7F10126EDE022A921229
:1029B0002AA57F10126EF1022A92E56B640270283C
:1029C000AF417802EF08800123D8FD3392307F2099
:1029D00020300A122A9A7F20126EDE8008122AA561
:1029E0007F20126EF1022A92E56B64037028AF41DA
:1029F0007801EF08800123D8FD3392307F402030EA
:102A00000A122AB07F40126EDE8008122ABB7F4075
:102A1000126EF1022A92E56B6404701EE541339256
:102A2000307F8020300A122AB07F80126EDE80084C
:102A3000122ABB7F80126EF18058E56B6405702707
:102A4000AF417805EF08800123D8FD3392307F0431
:102A500020300A122AC67F04126EDE8008122AD1A4
:102A60007F04126EF1802BE56B6406702CAF417809
:102A700004EF08800123D8FD3392307F0820300A0C
:102A8000122AC67F08126EDE8008122AD17F081231
:092A90006EF1AF6C7E00126C27A0
:102A990022126EF1AF6C7E00126C2722126EDEAF2D
:102AA9006C7E00126C2722126EF1AF6C7E00126CE4
:102AB9002722126EDEAF6C7E00126C2722126EF195
:102AC900AF6C7E00126C2722126EDEAF6C7E001294
:032AD9006C272245
:105D4B00900024E030E0057F10126EF1900024E00B
:105D5B0030E1057F20126EF1900024E030E2057FE8
:105D6B0040126EF1900024E030E3057F80126EF15B
:105D7B00900024E030E4057F04126EF1900024E0E3
:095D8B0030E5057F08126EF122DB
:106C930030030A124D02C203C211C21E223004097C
:0A6CA300124D02C204C213C21E22E9
:106517008F708D71E570B4011FE5717003125C6EA9
:10652700E571B401077880E6FF125A5CE571B43271
:106537000E7FF47E01026C27AD71AF7012665F2289
:10665F00EFFEEDFF1280008E2D8F2E12534B7574AF
:10666F0032AF741574EFD39400400EE4F573E573F5
:09667F00C3943A50EC057380F558
:0166880022EF
:10534B00D2A8AFA875A881C214852E82852D83E4BF
:10535B0093C4540FFE4306F08E80C284D28500C2E4
:10536B00870000D287007580FF7580FEC284C285DE
:10537B0000C2870000D287007580FFD2147D407C6D
:10538B001FE4FE30B40D0EBE32F9ED1D70011CEDA5
:10539B004C70EE7C1F7D40E4FE20B40D0EBE32F946
:1053AB00ED1D70011CED4C70EE8FA8C2A87F0A7E1C
:0453BB0000126C2749
:0153BF0022CB
:106689007580FDC284C28500C28700000000D287E0
:10669900007580FF7F0A7E00126C277F997E0912A0
:0A66A90080008E2D8F2E12534B221D
:10421100D284D285C286A2809217A2819220A282E4
:104221009218A2839221D2862001537D027F01122E
:104231004ED240137D037F01124ED2400A30170740
:10424100301932D22480377D027F01124ED2500FB5
:1042510030170C302009301904D224802180167DBA
:10426100037F01124ED2501220170330200C301957
:1042710004D22480091267568004C219C224200284
:104281004E7D027F02124ED240127D037F02124EFA
:10429100D24009301806301B2FD225227D027F0221
:1042A100124ED2500E30180B302108301B03D2258C
:1042B1002280157D037F02124ED2500F2018033049
:1042C1002109301B03D2252202677EC21BC225228F
:10675600753D1E753E60E4FFE53E2FF582E4353D4E
:10676600F583E4F00FBF50F0753D1E753E60E4F50D
:0767760045C226C211D21931
:01677D0022F9
:10677E00753F1E7540B0E4FFE5402FF582E4353FCE
:10678E00F583E4F00FBF10F0753F1E7540B0E4F5D1
:07679E0046C228C213D21B02
:0167A50022D1
:106BD100C284D285C286A2809209A281920AA2822F
:0D6BE100920BA283920DD286D284D285221F
:10611600E57E2560F582E4357DF5832274FF123A2B
:1061260020E4FBFAF9F8C3023A0D057F7480257E58
:10613600F57EE4357DF57D22F582E4341DF5832276
:0B614600757F01757D00757E20E4224E
:1042D1007D027F07124ED250057F04126EDEC22985
:1042E100D223E4F5427FE87E03126C27C298C2AF65
:1042F100C2307F03122EB6755E7F755D96755C9830
:10430100755B00785B126122504430983E120006C2
:10431100126DF4EF14601824F0602624C1600B24A0
:10432100F670287F06126F038021126200801C7FC5
:1043310006126F031269AF1264E7125DDCD22980A5
:104341000A7F06126F03125A0CD2293029B5E4787C
:1043510085F6D2307F01122EB67F40120016C22F91
:104361001269697D467F0212665F7D1E7F071266B4
:104371005F7D147F0812665F7D327F0312665FC224
:0D438100307F03122EB67FFF126E9DC22307
:01438E00220C
:105A0C00126146F55F7F02126F03E57F2402F56198
:105A1C00AF7F126F03E4F560126116E0FF126F03A3
:105A2C00126116E02561F5610560E560C394804064
:105A3C00E7AF61126F037F03126F03126F0BEF64FA
:0F5A4C0015600C126130055FE55FC3942240B610
:015A5B002228
:1069AF00126146F55F1266DC50077F06126F038097
:1069BF00057F15026F03126130055FE55FC39422F7
:0269CF0040E3A3
:0169D10022A3
:1066DC00E4F560126F0B74D0256012613EEFF0058B
:1066EC0060E560C3948440EB126DD2901E52E0B50D
:0866FC000705126C42D322C312
:016704002272
:106C4200E4FF74D22FF582E4341DF583E0FEE57E85
:0A6C52002F12611AEEF00FBF7FE869
:016C5C002215
:106DD200E4FFFE74D02E12613EE02FFF0EBE82F35E
:016DE200228E
:10620000E4F55FF5657564E0756393756204F561A7
:10621000786112612250213098F61200068F60E5F5
:106220006064046013AF65056574D02F12613EE5AC
:0862300060F0255FF55F80D8E6
:016238002243
:04000600AF99C29854
:01000A0022D3
:086F03003099FDC2998F99221B
:076F0B003098FDAF99C29818
:016F1200225C
:106CE0000C0102030405060708090A0B0C01020344
:086CF0000405060708090A0B60
:10670500AF5FEF3395E0FE75F007EF123A3EEE7599
:10671500F007A42583F583E0227883E6FF126CC792
:09672500EF22C295D297D2AF22F7
:10684200C22CC2AF126F137F83126CF8126AE0126D
:1068520067277884E66F600B125E64302B05125F47
:0568620068922CA22C3D
:01686700220E
:105F68007984E778876660367884E6FF7887F6EF85
:105F78007013E552C3940A500C7D077F04124ED269
:105F88005003125E217D057F04124ED25010E54168
:105F980054036005123FB3D322123FB3C322C32276
:103FB300E4F55F900A501267057003024077900A98
:103FC3005112670C60167881666003024077900A8D
:103FD300521267057888666003024077AF5FEF335C
:103FE30095E0FE900A5312670CFF7880E6FEEF6EB1
:103FF3006020EF601DB4080BEED394014005EE94EE
:1040030007400FEF6409706CEE64016005EE64070E
:104013007062AF5FEF3395E0FE900A5412670CFFB6
:10402300F46006EF788366704BE55FFD3395E0FC43
:10403300900A5575F007ED123A3EEC126714788436
:10404300667031D201D20274BD2DF58274003CF545
:1040530083E0FFC007EDAE047805C333CE33CED87B
:10406300F92480F582740E3EAD82FCD007125BD832
:10407300C201C202055FC3E55F64809493500302EB
:024083003FB646
:014085002218
:105E21007D087F04124ED2500D7883E6FF126CC7B5
:105E3100EFC39407402CD2307F01122EB67F40125F
:105E41000016C22F126969D201D202E4FD7F0A1243
:105E51004F5AC201C2027F50126E9DC2307F0112A1
:035E61002EB62238
:105E6400C2AF126F137FBF126CF8126AE07884A677
:105E740007126AE07884A607126AE07883A60712FC
:105E84006AE07888A607126AE07881A607126AE0B9
:105E94007880A607126AE07882A607126F13126749
:025EA4002722B3
:1057A500C2AF126F137F8E1257F47F90126CF87F81
:1057B500A7126CF8126F137FBE126CF8E4FF126C1F
:1057C500F87884E6FF126CF87883E6FF126CF878B7
:1057D50088E6FF126CF87881E6FF126CF87880E6AF
:1057E500FF126CF87882E6FF1257F412672722122F
:0B57F5006CF8E4FF126CF8126F132236
:105A5C008F72E572B401047D63803EE572B4020678
:105A6C007D087F068035E572B403067D317F0880A2
:105A7C002AE572B404067D617F08801FE572B405C7
:105A8C00067D257F088014E572B406067D597F03D8
:0F5A9C008009E572B407077D487F0712665F2215
:026CC700AE0716
:106CC900EE54F0FF780408800103D8FD75F00AA49A
:066CD900FFEE540F2FFF37
:016CDF002292
:105C6E0012671E906CE093FF1235A47884126720A1
:105C7E00601B7884126720C3940A50077D327F061A
:105C8E0012665F7884E6FF126CC71235A412671E87
:105C9E00C3940C50067D0A7F0280047D507F06124D
:0A5CAE00665F7D507F0512665F22DD
:105963007FF47E01126C277D097F0612665F7881C2
:105973001259A97D0E7F0312665F7D357F0612667D
:105983005F7D097F0612665F78881259A97D1E7FA5
:105993000912665F7D1E7F0712665F7882E6FF123B
:1059A3006CC71235A422E6FF126CC71235A47FF42C
:0659B3007E01126C2722A8
:076F1300C2B6C295D295221F
:106CF800E4FEC297EF30E002D297C2B6D2B6EFC335
:066D080013FF0EBE08ECB3
:016D0E002262
:106AE000E4FFD297FED2B6C2B6A297E433C43333E2
:0F6AF000335480FDEFC313FFED42070EBE08E6DF
:016AFF002274
:1056ED00EF3395E0FE74702FF58274003EF583E084
:1056FD00FF22AF5AEF3395E0FEEF222460F582745E
:10570D00013EAD82FCD22922900520E0F547A3E0B1
:10571D00F548222450F58274053EAD82FC2290009E
:10572D00BAE0FF7C0E7D2022D222D201E4FF22C2FC
:0D573D0001C2227F1922D222D2307F022227
:10281D00E5527008126EC78F52022918E552B405A1
:10282D000812438F8F52022918E552B40B08126C0F
:10283D005D8F52022918E552B40A08125CB88F5206
:10284D00022918E552B40F081260618F520229183F
:10285D00E552B414081223368F52022918E552B4EA
:10286D001908126B3D8F52022918E552B41E081239
:10287D006A188F52022918E552B42308126A7E8F06
:10288D0052022918E552B42807126EAB8F52807B85
:10289D00E552B42D071267CE8F52806FE552B432D8
:1028AD00071262398F528063E552B43E07126B5B9B
:1028BD008F528057E552B43C07126D9C8F52804B5E
:1028CD00E552B43307126A5C8F52803FE552B44132
:1028DD0007126E258F528033E552B44C07126E35B8
:1028ED008F528027E552B44407126E458F52801BDC
:1028FD00E552B4370712585A8F52800FE552B4394A
:10290D00071258008F528003E4F552E553700612FA
:10291D00000E8F5322E553B40506126EFA8F532223
:10292D00E553B40A06126E558F5322E553B40F06C4
:10293D00126E648F5322E553B41406123B5A8F5313
:10294D0022E553B43D06126B798F5322E553B43F04
:10295D00061265478F5322E553B443061267A68FBF
:10296D005322E553B44D06126A9F8F5322E4F5535B
:01297D002237
:0D6EC70090052AE0F52BA3E0F52C7F0522B5
:10438F00302414201011C21C7D047F01124ED25014
:10439F00037F0B227F0A227F0812631750061245F4
:1043AF00BB7F0022202408301005C2107F05227D1C
:1043BF00057F06124ED2501EE53945387018900011
:1043CF00B5E0FF7C0D7D80125BD890052EE0F538AF
:1043DF00A3E0F53980557D067F06124ED2501EE5BB
:1043EF003C453B70189000B6E0FF7C0D7DA0125B42
:1043FF00D8900530E0F53BA3E0F53C802E7D077F9C
:10440F0005124ED2500D30000AE52C452B7004C218
:10441F00008018300F0AE52C452B7004C20F800B5B
:10442F007885E6B405057F04125169E5517008756A
:0A443F00510AD22B1268427F0522B9
:106C5D00200F1590053BE0F54E2024037F0522E51E
:0B6C6D004ED3940050F3D20F7F0A2298
:105CB8007D077F05124ED2500C7D077F05124ED20C
:105CC800503230002F7D017F01124ED25026D23043
:105CD8007F01122EB67F011200167D027F07124E39
:105CE800D250057F04126EF19000A0E0FF7C0A7D7F
:0A5CF800E0125BD81257157F0F224F
:10606100302437E5484547700C7D087F01124ED238
:1060710050037F372230030EE53A700A126C937F8A
:106081000112001680113026037F14227885E6B4B0
:0D60910005057F031251697F0F227F142245
:1023360090053DE0F54B7F01126E9D126C937D0278
:102346007F07124ED25009E54B70057F04126EDEF0
:102356009000A1E0FF7C0B7D00125BD8D22B1268A7
:1023660042E54570030224607C017D001224DE50A4
:10237600037F3E227C017D501224BE50037F3C2207
:102386007C017D581224BE50037F3C227C017D10C7
:102396001224C650081224CE50037F33227C017DBE
:1023A600201224C6500B9000BBE0FF7C0E7D4080BF
:1023B600207C017D281224D6500512572B80127CD2
:1023C600017D301224D650129000B9E0FF7C0E7DBC
:1023D60000125BD81267567F00227C017D40D2290D
:1023E600E4FF1247D0500C7D067F04124ED25003F4
:1023F6007F4C227C017D381224DE50037F44227CF0
:10240600017D18C229E4FF1247D0500C7D057F01DB
:10241600124ED250037F4122E4F55A1256FF78033A
:10242600C333CE33CED8F9125708E4FF1247D05043
:102436001BAF5A1256EDC0071256FF7805C333CEAE
:1024460033CED8F9125720D007125B8D055AC3E553
:102456005A648094A840C47F19221224CE500C7D61
:10246600077F05124ED2504130003E7885E6700453
:102476007F0180087885E6B404077F0212516980DF
:10248600257D037F06124ED2501CE5574556701621
:102496009000AFE0FF7C0C7DC0125BD8900532E067
:1024A600F556A3E0F5577F19227D077F05124ED218
:0724B60050052000027F0524
:1024BD0022D229E4FF1247D022D229E4FF1247D0BD
:1024CD00227D077F05124ED222D229E4FF1247D07A
:0924DD0022C229E4FF1247D022BB
:106B3D003026031267567D077F05124ED250062070
:0E6B4D0000037F0522900538E0F54E7F1E22E2
:106A1800E54E70037F23227D027F07124ED2500974
:106A2800E54B70057F04126EDE3024037F0A227F57
:026A38001E221C
:106A7E001257157D067F01124ED2500C9000ACE0DD
:106A8E00FF7C0C7D60125BD8900539E0F54E7F2DB2
:016A9E0022D5
:0E6EAB007FA0126E9D900539E0F54E7F2D22DE
:1067CE00D22B1268427D027F07124ED25009E54B42
:1067DE0070057F04126EDEE54E70037F3222302488
:0767EE00037F0A227F2D2228
:10623900301E037F32227D047F06124ED2501FE5A5
:1062490055455470199000B0E0FF7C0C7DE0125B5D
:10625900D8900534E0F554A3E0F5557F3222C230D9
:086269007F01122EB67F002216
:106D9C0020220CD222E4FF12055BC2227F00227F4C
:026DAC003C2287
:106B5B00202218D2227F40120016D201121D7DC2B4
:0E6B6B00017F40126E9DC2227F19227F3E22C2
:106E250020220A12573512379F12573C227F4122E2
:106E350020220A1257351260DA12573C227F44226B
:106E450020220A12573512549C12573C227F4422A5
:05000E0000007F052247
:096EFA003025037F0A227F0522E6
:0F6E55009000A2E0FF7C0B7D20125BD87F0F2204
:0F6E64003025093028037F14227F0F227F14224C
:103B5A009000A3E0FF7C0B7D40125BD8E546700322
:103B6A00023C327D017F03124ED250707C017D08E7
:103B7A00C2297F011247D050037F3F227C017D502A
:103B8A00123C3550037F3D227C017D58123C355052
:103B9A00037F3D227C017D40D2297F011247D0500C
:103BAA000C7D067F04124ED250037F4D227C017D8C
:103BBA0028D2297F011247D0500912572B125BD8FD
:103BCA007F00227C017D18C2297F011247D0500C48
:103BDA007D057F02124ED250037F43227D027F036E
:103BEA00124ED25043E4F55AAF5A1257017803C322
:103BFA0033CE33CED8F91257087F011247D0501D61
:103C0A00AF5A1256EDC007AF5A1257017805C3339F
:103C1A00CE33CED8F9125720D007125B8D055AC37E
:0A3C2A00E55A648094A840C07F00B2
:093C340022D2297F011247D0229F
:106B7900202218D222C2307F01122EB67F01126E56
:0E6B89009D7F0112055BC2227F00227F3D220C
:1065470020222A125743122EB67FF47E01126C279F
:106557007F10120016D202121B7CC2027F10126E2D
:106567009DC2307F02122EB6C2227F00227F3F22B9
:1067A600202222125743122EB67FF47E01126C2746
:1067B600D2027F0112379FC202C2307F02122EB66A
:0867C600C2227F00227F432262
:106A9F0020221B125743122EB6D2027F011260DA48
:106AAF00C202C2307F02122EB6C2227F00227F4D59
:016ABF0022B4
:1055D000AF5AEF3395E0FE22900520E0F547A3E0B7
:1055E000F54822900522E0F549A3E0F54A2224601F
:1055F000F58274013EAD82FCD2292274702FF582AF
:1056000074003EF583E0FF22C202C2227F192224E9
:1056100050F58274053EAD82FC22055AC3E55A64FA
:105620008094A822D222C2307F0122D222C2307FAF
:02563000022254
:10325100E5527006126A3A8F5222E552B4050612FF
:1032610036A38F5222E552B40B061267F58F522214
:10327100E552B40A061244498F5222E552B40F06B0
:10328100126DAE8F5222E552B4110612590B8F52B4
:1032910022E552B412061251E38F5222E552B414C0
:1032A10006120A548F5222E552B419061265D68FBE
:1032B1005222E552B41E061265778F5222E552B4AE
:1032C1002306125EE78F5222E552B42806126EB928
:1032D1008F5222E552B42D061261518F5222E552CE
:1032E100B432061262718F5222E552B43C06126D5D
:1032F100C08F5222E552B43D06126C788F5222E5FE
:1033010052B43E061268D78F5222E552B43F0612DC
:103311006DE38F5222E552B44106126B008F5222A7
:10332100E552B443061269D28F5222E552B44C06DB
:10333100126CAD8F5222E552B44D061269F58F52CF
:1033410022E552B4370612585A8F5222E552B43947
:10335100061258008F5222E552B438061268FC8FCB
:103361005222E552B43306126A5C8F5222E552B4FE
:0C3371004406126D0F8F5222E4F5522228
:106A3A0090052AE0F52BA3E0F52C7D067F02124E85
:106A4A00D2500C90052CE0F529A3E0F52AD21F7F3D
:026A5A00052213
:1036A300302414201011C21C7D047F01124ED2500D
:1036B300037F0B227F0A22302514201211D21C7D96
:1036C300047F02124ED250037F0B227F0A227F080F
:1036D30012631750061245BB7F00222024083010C6
:1036E30005C2107F0522202508301205C2127F056E
:1036F300227D057F06124ED2501EE53945387018DB
:103703009000B5E0FF7C0D7D80125BD890052EE024
:10371300F538A3E0F53980757D067F06124ED25049
:103723001EE53C453B70189000B6E0FF7C0D7DA084
:10373300125BD8900530E0F53BA3E0F53C804E7D6D
:10374300077F05124ED2500D30000AE52C452B7031
:1037530004C200800B300F08E52C452B7002C20F0A
:103763007D067F02124ED25019301F16E52A4529D5
:103773007010C21F9000BCE0FF7C0E7D60125BD80E
:10378300800B7885E6B405057F04125169E5517015
:0C3793000875510AD22B1268427F0522F3
:1067F500200F2190053BE0F54E202406201C037F49
:106805000522202506301C037F0522E54ED3940082
:0768150050E7D20F7F0A22B9
:104449007D077F05124ED250127D077F05124ED28D
:1044590040030244FA2000030244FA201C3FD230F0
:104469007F03122EB67F0F126E9D90000FE0B402EB
:10447900047F05800990000FE0B403057F01120055
:10448900161255D87D027F07124ED250057F0412AD
:104499006EF19000A0E0FF7C0A7DE0804E301C5157
:1044A90090000FE0FF64026005EF640370437F0F23
:1044B900126E9D7F05126317400BD2307F01122EB9
:1044C900B67F028009D2307F03122EB67F0A12000E
:1044D900167D027F07124ED250057F04126EF1122B
:1044E90055E39000A2E0FF7C0B7D20125BD87F0F83
:0A44F900221255D81255E37F0F225E
:106DAE00201C063024037F1122301C053025027F63
:026DBE0012229F
:10590B00302452E5484547700C7D087F01124ED27A
:10591B0050037F3722300329E53A70257FA0126EA2
:10592B009D90000FE0B401047F01800990000FE00F
:10593B00B402057F05120016E4F542C21EC20380B5
:10594B00113026037F14227885E6B405057F0312F8
:08595B0051697F11227F142223
:1051E300301C1030240D20100A7F0A126E9DC21C41
:1051F3007F0A22301C4C302549201246300303120B
:105203006C93E54A4549700C7D087F02124ED250DB
:10521300037F3822300417E53A70137FA0126E9D86
:105223007F02120016E4F542C21EC2048011302828
:10523300037F14227885E6B405057F031251697F45
:105243001222201C1230250F20120CD21CC2307FD8
:0A52530002122EB67F0A227F1422F9
:100A540090053DE0F54B7F0F126E9D201C0C90001D
:100A6400A1E0FF7C0B7D00125BD8301C0C9000A32E
:100A7400E0FF7C0B7D40125BD8E542B403037F1496
:100A840022126C93E4F5427D027F07124ED2500984
:100A9400E54B70057F04126EDED22B126842301CC7
:100AA40003020B97E5457003020B977C017D00124E
:100AB4000D1450037F3E227C017D50120CE4500340
:100AC4007F3C227C017D58120CE450037F3C227C45
:100AD400017D10120CEC5008120CFC50037F3322E1
:100AE4007C017D20120CEC5003020BFE7C017D285E
:100AF400120D04500C9000BAE0FF7C0E7D20020C15
:100B0400077C017D30120D04500C9000B9E0FF7C8D
:100B14000E7D00020C077C017D40D229E4FF1247C0
:100B2400D0500C7D067F04124ED250037F4C227CA1
:100B3400017D38120D1450037F44227C017D18C2BC
:100B440029E4FF1247D0500C7D057F01124ED2508C
:100B5400037F4122E4F55A1255D0EF7803C333CE14
:100B640033CED8F91255EEE4FF1247D0501D12557A
:100B7400D01255FBC0071255D0EF7805C333CE33DE
:100B8400CED8F912560FD007125B8D12561A40C7F1
:100B94007F1922201C03020C8AE5467003020C8A8A
:100BA4007D017F03124ED24003020C427C017D087A
:100BB400C2297F011247D0500F7F50120016D23045
:100BC4007F02122EB67F3F227C017D50120CF4501E
:100BD400037F3D227C017D58120CF450037F3D229B
:100BE4007C017D10120D0C5008120CFC50037F3355
:100BF400227C017D20120D0C50129000BBE0FF7C82
:100C04000E7D40125BD81267567F00227C017D4026
:100C1400D2297F011247D0500C7D067F04124ED298
:100C240050037F4D227C017D18C2297F011247D0D9
:100C3400500C7D057F02124ED250037F43227D0269
:100C44007F03124ED2503CE4F55A1255D0EF78038C
:100C5400C333CE33CED8F91255EE7F011247D050AC
:100C64001D1255D01255FBC0071255D0EF7805C39D
:100C740033CE33CED8F912560FD007125B8D1256ED
:100C84001A40C77F1922120D1C5008120D1C504126
:100C940030003E7885E670047F0180087885E6B4EC
:100CA40004077F0212516980257D037F06124ED20C
:100CB400501CE557455670169000AFE0FF7C0C7D44
:100CC400C0125BD8900532E0F556A3E0F5577F19C2
:0F0CD400227D077F05124ED250052000027F05BA
:100CE30022D229E4FF1247D022D229E4FF1247D0AF
:100CF30022D2297F011247D0227D077F05124ED2CF
:100D030022D229E4FF1247D022D2297F011247D0F1
:100D130022C229E4FF1247D0227D077F05124ED25B
:010D230022AD
:1065D600C219C2307F02122EB630260512675680C7
:1065E6000630280312677E7D077F05124ED25006BD
:0F65F6002000037F0522900538E0F54E7F1E221E
:10657700E54E70037F23227D027F07124ED250091A
:10658700E54B70057F04126EDE3024062010037F72
:106597000A22302508201205D21C7F0A227F1E22DC
:105EE700201C051255D880031255E37D067F011249
:105EF7004ED25024E5427020201C0B9000ACE0FFEE
:105F07007C0C7D60800C301C0C9000ADE0FF7C0C9D
:105F17007D80125BD87F2822900539E0F54E7F2DD2
:015F27002257
:0E6EB9007FA0126E9D900539E0F54E7F2D22D0
:10615100D22B1268427D027F07124ED25009E54BC5
:1061610070057F04126EDEE54E601D30240620109E
:10617100037F0A2290000FE06401600930250620A8
:0B61810012037F05227F2D227F3222B7
:10627100301E037F32227D047F06124ED2501FE56D
:1062810055455470199000B0E0FF7C0C7DE0125B25
:10629100D8900534E0F554A3E0F5557F3222C230A1
:0862A1007F01122EB67F0022DE
:106DC00020220CD222E4FF12055BC2227F00227F28
:026DD0003C2263
:1068D70020221FC2307F02122EB6D2227F40120022
:1068E70016D201121D7DC2017F40126E9DC2227F0A
:0568F70019227F3E2282
:106DE30020220BD222D202121B7C125608227F3F92
:016DF300227D
:106C7800202215125624122EB67F40126E9D7F01D7
:0B6C880012055BC2227F00227F3D222C
:106B000020221912562B122EB67F10126E9DD20122
:0F6B1000E4FF12379FC201C2227F19227F412268
:1069D20020221D125624122EB67F40126E9DD230F6
:1069E2007F02122EB6D2027F0112379F1256082260
:0369F2007F4322BE
:106CAD0020221412562B122EB6D201E4FF1260DAF6
:0A6CBD00C201C2227F19227F41228A
:1069F50020221D125624122EB67F40126E9DD230D3
:106A05007F02122EB6D2027F011260DA12560822D8
:036A15007F43229A
:106D0F0020221112562B122EB6D202E4FF12549CDF
:076D1F00125608227F4422F6
:10585A00D2107D027F07124ED250057F04126EDEEF
:10586A0090000FE0FF64016004EFB4030E7F0112A1
:10587A006E9D7F401258A37F01801390000FE0B401
:10588A00020F7F05126E9D7F501258A37F03126E7E
:10589A00DE7F50126E9D7F3922120016C22F1269C6
:0958AA0069E4FD7F07124F5A2248
:105800003024037F3922E47885F6C21090000FE03F
:10581000FF64016004EFB4030E7F01126EF17F405C
:1058200012584A7F01801890000FE0B402147F03E1
:10583000126EF17F05126E9D7F5012584A7F03123F
:105840006EDE7F50126E9D7F0022120016C22F1254
:0A5850006969E4FD7F08124F5A2237
:1068FC00D2127F0A126E9D7F40120016D22F12699F
:10690C0069E4FD7F07124F5A7F03126EDE7F50122F
:05691C006E9D7F0022CA
:106A5C0030000B9000B8E0FF7C0D7DE0800C200036
:106A6C000E9000B7E0FF7C0D7DC0125BD8B2007FAA
:026A7C001922DD
:1060DA008F5AE55A24FF922F126969E55A70127F86
:1060EA0040120016D201E4FD7F09124F5AC2018004
:1060FA0015E55AB401107F10120016D202E4FD7F92
:0C610A0009124F5AC2027F50126E9D22F3
:104D2B00C201C202D20C7F50126E9D7F8012001600
:104D3B0075420390000FE0B401163024647F01121A
:104D4B000016302407E542D3940050F67F01804EC5
:104D5B0090000FE0FF64026005EF640370433024A2
:104D6B00267F02126E9DD2307F03122EB67F051264
:104D7B000016302407E542D3940050F6C2307F0270
:104D8B00122EB67F0580173025177F0212001630C2
:104D9B00250AE542D3940040033024F37F02126EC0
:0F4DAB009DE542708E7FA0126E9DC20CC21E222B
:03000000026BEEA2
:106BEE00758E0078FEE4F6D8FD9000007FFF7E1FC4
:0D6BFE00E4F0A3DFFCDEFA758188024C0C88
:10398400C2D530F707B2D563F0FF05F030E70CB2CB
:10399400D5F4048463F0FF05F080018430D502F48B
:0239A4000422FB
:1039A600EF8DF0A4A8F0CF8CF0A428CE8DF0A42E35
:0239B600FE22EF
:1039B800BC000BBE0029EF8DF084FFADF022E4CCF3
:1039C800F875F008EF2FFFEE33FEEC33FCEE9DECBC
:1039D800984005FCEE9DFE0FD5F0E9E4CEFD22ED02
:1039E800F8F5F0EE8420D21CFEADF075F008EF2F4C
:1039F800FFED33FD4007985006D5F0F222C398FD3D
:053A08000FD5F0EA22D9
:103A0D00EB9FF5F0EA9E42F0E99D42F0E89C45F00F
:013A1D002286
:103A1E007401FF3395E0FEFDFC080808E6CF2FF693
:103A2E0018E6CE3EF618E6CD3DF618E6CC3CF6226C
:0C3A3E00A42582F582E5F03583F5832293
:103A4A00D083D082F8E4937012740193700DA3A30B
:103A5A0093F8740193F5828883E47374029368601F
:063A6A00EFA3A3A380DF1F
:106DF400EFC39461400AEF947B5005EF24E0FF2237
:016E0400226B
:00000001FF
